 jaccesswalker

 Timestamp is da4eb605 (reproducible build file hash)

 Preferred load address is 0000000140000000

 Start         Length     Name                   Class
 0001:00000000 00008870H .text$mn                CODE
 0001:00008870 00000040H .text$mn$00             CODE
 0001:000088b0 00000053H .text$x                 CODE
 0002:00000000 000003a0H .idata$5                DATA
 0002:000003a0 00000038H .00cfg                  DATA
 0002:000003d8 00000008H .CRT$XCA                DATA
 0002:000003e0 00000008H .CRT$XCAA               DATA
 0002:000003e8 00000008H .CRT$XCZ                DATA
 0002:000003f0 00000008H .CRT$XIA                DATA
 0002:000003f8 00000008H .CRT$XIAA               DATA
 0002:00000400 00000008H .CRT$XIAC               DATA
 0002:00000408 00000008H .CRT$XIZ                DATA
 0002:00000410 00000008H .CRT$XPA                DATA
 0002:00000418 00000008H .CRT$XPZ                DATA
 0002:00000420 00000008H .CRT$XTA                DATA
 0002:00000428 00000008H .CRT$XTZ                DATA
 0002:00000430 00000000H .gehcont$y              DATA
 0002:00000430 00000000H .gfids$y                DATA
 0002:00000430 00001d50H .rdata                  DATA
 0002:00002180 00000000H .rdata$CastGuardVftablesA DATA
 0002:00002180 00000000H .rdata$CastGuardVftablesC DATA
 0002:00002180 000001f4H .rdata$r                DATA
 0002:00002374 000000b0H .rdata$voltmd           DATA
 0002:00002424 0000033cH .rdata$zzzdbg           DATA
 0002:00002760 00000008H .rtc$IAA                DATA
 0002:00002768 00000008H .rtc$IZZ                DATA
 0002:00002770 00000008H .rtc$TAA                DATA
 0002:00002778 00000008H .rtc$TZZ                DATA
 0002:00002780 000005c0H .xdata                  DATA
 0002:00002d40 000000ecH .xdata$x                DATA
 0002:00002e2c 00000000H .edata                  DATA
 0002:00002e2c 00000118H .idata$2                DATA
 0002:00002f44 00000014H .idata$3                DATA
 0002:00002f58 000003a0H .idata$4                DATA
 0002:000032f8 00000882H .idata$6                DATA
 0003:00000000 00000bd8H .data                   DATA
 0003:00000bd8 00000080H .data$r                 DATA
 0003:00000c58 00000028H .data$rs                DATA
 0003:00000c80 00000ae0H .bss                    DATA
 0004:00000000 00000888H .pdata                  DATA
 0005:00000000 000001d0H .rsrc$01                DATA
 0005:000001d0 00000558H .rsrc$02                DATA

  Address         Publics by Value              Rva+Base               Lib:Object

 0000:00000000       __AbsoluteZero             0000000000000000     <absolute>
 0000:00000000       ___safe_se_handler_count   0000000000000000     <absolute>
 0000:00000000       ___safe_se_handler_table   0000000000000000     <absolute>
 0000:00000000       __arm64x_extra_rfe_table   0000000000000000     <absolute>
 0000:00000000       __arm64x_extra_rfe_table_size 0000000000000000     <absolute>
 0000:00000000       __arm64x_native_entrypoint 0000000000000000     <absolute>
 0000:00000000       __arm64x_redirection_metadata 0000000000000000     <absolute>
 0000:00000000       __arm64x_redirection_metadata_count 0000000000000000     <absolute>
 0000:00000000       __dynamic_value_reloc_table 0000000000000000     <absolute>
 0000:00000000       __enclave_config           0000000000000000     <absolute>
 0000:00000000       __guard_check_icall_a64n_fptr 0000000000000000     <absolute>
 0000:00000000       __guard_eh_cont_count      0000000000000000     <absolute>
 0000:00000000       __guard_eh_cont_table      0000000000000000     <absolute>
 0000:00000000       __guard_fids_count         0000000000000000     <absolute>
 0000:00000000       __guard_fids_table         0000000000000000     <absolute>
 0000:00000000       __guard_iat_count          0000000000000000     <absolute>
 0000:00000000       __guard_iat_table          0000000000000000     <absolute>
 0000:00000000       __guard_longjmp_count      0000000000000000     <absolute>
 0000:00000000       __guard_longjmp_table      0000000000000000     <absolute>
 0000:00000000       __hybrid_auxiliary_delayload_iat 0000000000000000     <absolute>
 0000:00000000       __hybrid_auxiliary_delayload_iat_copy 0000000000000000     <absolute>
 0000:00000000       __hybrid_auxiliary_iat     0000000000000000     <absolute>
 0000:00000000       __hybrid_auxiliary_iat_copy 0000000000000000     <absolute>
 0000:00000000       __hybrid_code_map          0000000000000000     <absolute>
 0000:00000000       __hybrid_code_map_count    0000000000000000     <absolute>
 0000:00000000       __hybrid_image_info_bitfield 0000000000000000     <absolute>
 0000:00000000       __x64_code_ranges_to_entry_points 0000000000000000     <absolute>
 0000:00000000       __x64_code_ranges_to_entry_points_count 0000000000000000     <absolute>
 0000:00000100       __guard_flags              0000000000000100     <absolute>
 0000:00000000       __ImageBase                0000000140000000     <linker-defined>
 0001:00000000       initializeAccessBridge     0000000140001000 f   AccessBridgeCalls.obj
 0001:000010d0       shutdownAccessBridge       00000001400020d0 f   AccessBridgeCalls.obj
 0001:00001120       IsJavaWindow               0000000140002120 f   AccessBridgeCalls.obj
 0001:00001160       GetAccessibleContextFromHWND 0000000140002160 f   AccessBridgeCalls.obj
 0001:000011a0       getHWNDFromAccessibleContext 00000001400021a0 f   AccessBridgeCalls.obj
 0001:000011e0       SetJavaShutdown            00000001400021e0 f   AccessBridgeCalls.obj
 0001:00001210       SetFocusGained             0000000140002210 f   AccessBridgeCalls.obj
 0001:00001240       SetFocusLost               0000000140002240 f   AccessBridgeCalls.obj
 0001:00001270       SetCaretUpdate             0000000140002270 f   AccessBridgeCalls.obj
 0001:000012a0       SetMouseClicked            00000001400022a0 f   AccessBridgeCalls.obj
 0001:000012d0       SetMouseEntered            00000001400022d0 f   AccessBridgeCalls.obj
 0001:00001300       SetMouseExited             0000000140002300 f   AccessBridgeCalls.obj
 0001:00001330       SetMousePressed            0000000140002330 f   AccessBridgeCalls.obj
 0001:00001360       SetMouseReleased           0000000140002360 f   AccessBridgeCalls.obj
 0001:00001390       SetMenuCanceled            0000000140002390 f   AccessBridgeCalls.obj
 0001:000013c0       SetMenuDeselected          00000001400023c0 f   AccessBridgeCalls.obj
 0001:000013f0       SetMenuSelected            00000001400023f0 f   AccessBridgeCalls.obj
 0001:00001420       SetPopupMenuCanceled       0000000140002420 f   AccessBridgeCalls.obj
 0001:00001450       SetPopupMenuWillBecomeInvisible 0000000140002450 f   AccessBridgeCalls.obj
 0001:00001480       SetPopupMenuWillBecomeVisible 0000000140002480 f   AccessBridgeCalls.obj
 0001:000014b0       SetPropertyNameChange      00000001400024b0 f   AccessBridgeCalls.obj
 0001:000014e0       SetPropertyDescriptionChange 00000001400024e0 f   AccessBridgeCalls.obj
 0001:00001510       SetPropertyStateChange     0000000140002510 f   AccessBridgeCalls.obj
 0001:00001540       SetPropertyValueChange     0000000140002540 f   AccessBridgeCalls.obj
 0001:00001570       SetPropertySelectionChange 0000000140002570 f   AccessBridgeCalls.obj
 0001:000015a0       SetPropertyTextChange      00000001400025a0 f   AccessBridgeCalls.obj
 0001:000015d0       SetPropertyCaretChange     00000001400025d0 f   AccessBridgeCalls.obj
 0001:00001600       SetPropertyVisibleDataChange 0000000140002600 f   AccessBridgeCalls.obj
 0001:00001630       SetPropertyChildChange     0000000140002630 f   AccessBridgeCalls.obj
 0001:00001660       SetPropertyActiveDescendentChange 0000000140002660 f   AccessBridgeCalls.obj
 0001:00001690       SetPropertyTableModelChange 0000000140002690 f   AccessBridgeCalls.obj
 0001:000016c0       ReleaseJavaObject          00000001400026c0 f   AccessBridgeCalls.obj
 0001:000016f0       GetVersionInfo             00000001400026f0 f   AccessBridgeCalls.obj
 0001:00001730       GetAccessibleContextAt     0000000140002730 f   AccessBridgeCalls.obj
 0001:00001790       GetAccessibleContextWithFocus 0000000140002790 f   AccessBridgeCalls.obj
 0001:000017d0       GetAccessibleContextInfo   00000001400027d0 f   AccessBridgeCalls.obj
 0001:00001810       GetAccessibleChildFromContext 0000000140002810 f   AccessBridgeCalls.obj
 0001:00001850       GetAccessibleParentFromContext 0000000140002850 f   AccessBridgeCalls.obj
 0001:00001890       GetAccessibleTextInfo      0000000140002890 f   AccessBridgeCalls.obj
 0001:000018e0       GetAccessibleTextItems     00000001400028e0 f   AccessBridgeCalls.obj
 0001:00001930       GetAccessibleTextSelectionInfo 0000000140002930 f   AccessBridgeCalls.obj
 0001:00001970       GetAccessibleTextAttributes 0000000140002970 f   AccessBridgeCalls.obj
 0001:000019c0       GetAccessibleTextRect      00000001400029c0 f   AccessBridgeCalls.obj
 0001:00001a10       GetAccessibleTextLineBounds 0000000140002a10 f   AccessBridgeCalls.obj
 0001:00001a70       GetAccessibleTextRange     0000000140002a70 f   AccessBridgeCalls.obj
 0001:00001ad0       getAccessibleTableInfo     0000000140002ad0 f   AccessBridgeCalls.obj
 0001:00001b10       getAccessibleTableCellInfo 0000000140002b10 f   AccessBridgeCalls.obj
 0001:00001b70       getAccessibleTableRowHeader 0000000140002b70 f   AccessBridgeCalls.obj
 0001:00001bb0       getAccessibleTableColumnHeader 0000000140002bb0 f   AccessBridgeCalls.obj
 0001:00001bf0       getAccessibleTableRowDescription 0000000140002bf0 f   AccessBridgeCalls.obj
 0001:00001c30       getAccessibleTableColumnDescription 0000000140002c30 f   AccessBridgeCalls.obj
 0001:00001c70       getAccessibleTableRowSelectionCount 0000000140002c70 f   AccessBridgeCalls.obj
 0001:00001cb0       isAccessibleTableRowSelected 0000000140002cb0 f   AccessBridgeCalls.obj
 0001:00001cf0       getAccessibleTableRowSelections 0000000140002cf0 f   AccessBridgeCalls.obj
 0001:00001d40       getAccessibleTableColumnSelectionCount 0000000140002d40 f   AccessBridgeCalls.obj
 0001:00001d80       isAccessibleTableColumnSelected 0000000140002d80 f   AccessBridgeCalls.obj
 0001:00001dc0       getAccessibleTableColumnSelections 0000000140002dc0 f   AccessBridgeCalls.obj
 0001:00001e10       getAccessibleTableRow      0000000140002e10 f   AccessBridgeCalls.obj
 0001:00001e60       getAccessibleTableColumn   0000000140002e60 f   AccessBridgeCalls.obj
 0001:00001eb0       getAccessibleTableIndex    0000000140002eb0 f   AccessBridgeCalls.obj
 0001:00001f00       getAccessibleRelationSet   0000000140002f00 f   AccessBridgeCalls.obj
 0001:00001f40       getAccessibleHypertext     0000000140002f40 f   AccessBridgeCalls.obj
 0001:00001f80       activateAccessibleHyperlink 0000000140002f80 f   AccessBridgeCalls.obj
 0001:00001fc0       getAccessibleHyperlinkCount 0000000140002fc0 f   AccessBridgeCalls.obj
 0001:00002000       getAccessibleHypertextExt  0000000140003000 f   AccessBridgeCalls.obj
 0001:00002050       getAccessibleHypertextLinkIndex 0000000140003050 f   AccessBridgeCalls.obj
 0001:000020a0       getAccessibleHyperlink     00000001400030a0 f   AccessBridgeCalls.obj
 0001:000020f0       getAccessibleKeyBindings   00000001400030f0 f   AccessBridgeCalls.obj
 0001:00002130       getAccessibleIcons         0000000140003130 f   AccessBridgeCalls.obj
 0001:00002170       getAccessibleActions       0000000140003170 f   AccessBridgeCalls.obj
 0001:000021b0       doAccessibleActions        00000001400031b0 f   AccessBridgeCalls.obj
 0001:00002200       IsSameObject               0000000140003200 f   AccessBridgeCalls.obj
 0001:00002240       setTextContents            0000000140003240 f   AccessBridgeCalls.obj
 0001:00002280       getParentWithRole          0000000140003280 f   AccessBridgeCalls.obj
 0001:000022c0       getParentWithRoleElseRoot  00000001400032c0 f   AccessBridgeCalls.obj
 0001:00002300       getTopLevelObject          0000000140003300 f   AccessBridgeCalls.obj
 0001:00002340       getObjectDepth             0000000140003340 f   AccessBridgeCalls.obj
 0001:00002380       getActiveDescendent        0000000140003380 f   AccessBridgeCalls.obj
 0001:000023c0       GetCurrentAccessibleValueFromContext 00000001400033c0 f   AccessBridgeCalls.obj
 0001:00002410       GetMaximumAccessibleValueFromContext 0000000140003410 f   AccessBridgeCalls.obj
 0001:00002460       GetMinimumAccessibleValueFromContext 0000000140003460 f   AccessBridgeCalls.obj
 0001:000024b0       GetAccessibleSelectionFromContext 00000001400034b0 f   AccessBridgeCalls.obj
 0001:000024f0       GetAccessibleSelectionCountFromContext 00000001400034f0 f   AccessBridgeCalls.obj
 0001:00002530       IsAccessibleChildSelectedFromContext 0000000140003530 f   AccessBridgeCalls.obj
 0001:00002570       RemoveAccessibleSelectionFromContext 0000000140003570 f   AccessBridgeCalls.obj
 0001:000025b0       SelectAllAccessibleSelectionFromContext 00000001400035b0 f   AccessBridgeCalls.obj
 0001:000025e0       getVirtualAccessibleName   00000001400035e0 f   AccessBridgeCalls.obj
 0001:00002630       requestFocus               0000000140003630 f   AccessBridgeCalls.obj
 0001:00002670       selectTextRange            0000000140003670 f   AccessBridgeCalls.obj
 0001:000026c0       getTextAttributesInRange   00000001400036c0 f   AccessBridgeCalls.obj
 0001:00002720       getVisibleChildrenCount    0000000140003720 f   AccessBridgeCalls.obj
 0001:00002760       getVisibleChildren         0000000140003760 f   AccessBridgeCalls.obj
 0001:000027b0       setCaretPosition           00000001400037b0 f   AccessBridgeCalls.obj
 0001:000027f0       getCaretLocation           00000001400037f0 f   AccessBridgeCalls.obj
 0001:00002840       getEventsWaiting           0000000140003840 f   AccessBridgeCalls.obj
 0001:00002870       addAccessibleSelectionFromContext 0000000140003870 f   AccessBridgeCalls.obj
 0001:000028b0       clearAccessibleSelectionFromContext 00000001400038b0 f   AccessBridgeCalls.obj
 0001:000028e0       printError                 00000001400038e0 f   AccessBridgeDebug.obj
 0001:00002a30       PrintDebugString           0000000140003a30 f   AccessBridgeDebug.obj
 0001:00002ac0       wPrintJavaDebugString      0000000140003ac0 f   AccessBridgeDebug.obj
 0001:00002b50       wPrintDebugString          0000000140003b50 f   AccessBridgeDebug.obj
 0001:00002be0       initializeFileLogger       0000000140003be0 f   AccessBridgeDebug.obj
 0001:00002d60       finalizeFileLogger         0000000140003d60 f   AccessBridgeDebug.obj
 0001:00002da0       getTimeStamp               0000000140003da0 f   AccessBridgeDebug.obj
 0001:00002df0       PrintJavaDebugString2      0000000140003df0 f   AccessBridgeDebug.obj
 0001:00002e70       __local_stdio_printf_options 0000000140003e70 f i AccessBridgeDebug.obj
 0001:00002e80       _vfprintf_l                0000000140003e80 f i AccessBridgeDebug.obj
 0001:00002ed0       _vfwprintf_l               0000000140003ed0 f i AccessBridgeDebug.obj
 0001:00002f20       fprintf                    0000000140003f20 f i AccessBridgeDebug.obj
 0001:00002f70       printf                     0000000140003f70 f i AccessBridgeDebug.obj
 0001:00002fd0       vfprintf                   0000000140003fd0 f i AccessBridgeDebug.obj
 0001:00003000       vfwprintf                  0000000140004000 f i AccessBridgeDebug.obj
 0001:00003030       ?initBroadcastMessageIDs@@YAHXZ 0000000140004030 f   AccessBridgeMessages.obj
 0001:00003080       ?getTimeAndDate@@YAPEADXZ  0000000140004080 f   AccessInfo.obj
 0001:00003150       ?displayAndLog@@YAXPEAUHWND__@@HPEAU_iobuf@@PEADZZ 0000000140004150 f   AccessInfo.obj
 0001:00003270       ?logString@@YAXPEAU_iobuf@@PEBDZZ 0000000140004270 f   AccessInfo.obj
 0001:00003330       ?getAccessibleInfo@@YAPEADJ_JPEADH@Z 0000000140004330 f   AccessInfo.obj
 0001:00003380       ?getAccessibleInfo@@YAPEADJ_JHHPEADH@Z 0000000140004380 f   AccessInfo.obj
 0001:00005d60       ?appendToBuffer@@YAHPEAD_KPEBDZZ 0000000140006d60 f   AccessInfo.obj
 0001:00005e70       snprintf                   0000000140006e70 f i AccessInfo.obj
 0001:00005ed0       vsnprintf                  0000000140006ed0 f i AccessInfo.obj
 0001:00005f50       WinMain                    0000000140006f50 f   jaccesswalker.obj
 0001:00006010       ??0AccessibleNode@@QEAA@J_JPEAV0@PEAUHWND__@@PEAU_TREEITEM@@@Z 0000000140007010 f   jaccesswalker.obj
 0001:00006080       ??1AccessibleNode@@QEAA@XZ 0000000140007080 f   jaccesswalker.obj
 0001:000060b0       ?setAccessibleName@AccessibleNode@@QEAAXPEAD@Z 00000001400070b0 f   jaccesswalker.obj
 0001:000060f0       ?setAccessibleRole@AccessibleNode@@QEAAXPEAD@Z 00000001400070f0 f   jaccesswalker.obj
 0001:00006130       ?displayAPIWindow@AccessibleNode@@QEAAHXZ 0000000140007130 f   jaccesswalker.obj
 0001:00006290       ??0Jaccesswalker@@QEAA@H@Z 0000000140007290 f   jaccesswalker.obj
 0001:00006540       ?buildAccessibilityTree@Jaccesswalker@@QEAAXXZ 0000000140007540 f   jaccesswalker.obj
 0001:00006580       ?addComponentNodes@Jaccesswalker@@QEAAXJ_JPEAVAccessibleNode@@PEAUHWND__@@PEAU_TREEITEM@@2@Z 0000000140007580 f   jaccesswalker.obj
 0001:000068d0       ?WinProc@@YA_JPEAUHWND__@@I_K_J@Z 00000001400078d0 f   jaccesswalker.obj
 0001:00006be0       ?EnumWndProc@@YAHPEAUHWND__@@_J@Z 0000000140007be0 f   jaccesswalker.obj
 0001:00006d10       ?EnumChildProc@@YAHPEAUHWND__@@_J@Z 0000000140007d10 f   jaccesswalker.obj
 0001:00006dd0       ?CreateATreeView@@YAPEAUHWND__@@PEAU1@@Z 0000000140007dd0 f   jaccesswalker.obj
 0001:00006e90       ?AccessInfoWindowProc@@YA_JPEAUHWND__@@IIJ@Z 0000000140007e90 f   jaccesswalker.obj
 0001:00007050       ?IsInaccessibleJavaWindow@@YAHQEAUHWND__@@@Z 0000000140008050 f   jaccesswalker.obj
 0001:000076dc       ??_U@YAPEAX_K@Z            00000001400086dc f   MSVCRT:new_array.obj
 0001:000076e4       ??3@YAXPEAX_K@Z            00000001400086e4 f   MSVCRT:delete_scalar_size.obj
 0001:000076e4       ??_V@YAXPEAX@Z             00000001400086e4 f   MSVCRT:delete_array.obj
 0001:000076ec       __raise_securityfailure    00000001400086ec f   MSVCRT:gs_report.obj
 0001:00007720       __report_gsfailure         0000000140008720 f   MSVCRT:gs_report.obj
 0001:000077f4       __report_rangecheckfailure 00000001400087f4 f   MSVCRT:gs_report.obj
 0001:00007808       __report_securityfailure   0000000140008808 f   MSVCRT:gs_report.obj
 0001:00007988       __GSHandlerCheck           0000000140008988 f   MSVCRT:gshandler.obj
 0001:000079a8       __GSHandlerCheckCommon     00000001400089a8 f   MSVCRT:gshandler.obj
 0001:00007a20       __chkstk                   0000000140008a20 f   MSVCRT:chkstk.obj
 0001:00007a20       _alloca_probe              0000000140008a20 f   MSVCRT:chkstk.obj
 0001:00007a80       __security_check_cookie    0000000140008a80 f   MSVCRT:amdsecgs.obj
 0001:00007aa0       ??2@YAPEAX_K@Z             0000000140008aa0 f   MSVCRT:new_scalar.obj
 0001:00007adc       __GSHandlerCheck_EH4       0000000140008adc f   MSVCRT:gshandlereh4.obj
 0001:00007db4       WinMainCRTStartup          0000000140008db4 f   MSVCRT:exe_winmain.obj
 0001:00007dc8       ??3@YAXPEAX@Z              0000000140008dc8 f   MSVCRT:delete_scalar.obj
 0001:00007dd0       ??0bad_alloc@std@@QEAA@AEBV01@@Z 0000000140008dd0 f i MSVCRT:throw_bad_alloc.obj
 0001:00007e0c       ??0bad_alloc@std@@QEAA@XZ  0000000140008e0c f i MSVCRT:throw_bad_alloc.obj
 0001:00007e2c       ??0bad_array_new_length@std@@QEAA@AEBV01@@Z 0000000140008e2c f i MSVCRT:throw_bad_alloc.obj
 0001:00007e68       ??0bad_array_new_length@std@@QEAA@XZ 0000000140008e68 f i MSVCRT:throw_bad_alloc.obj
 0001:00007e88       ??0exception@std@@QEAA@AEBV01@@Z 0000000140008e88 f i MSVCRT:throw_bad_alloc.obj
 0001:00007ebc       ??1bad_alloc@std@@UEAA@XZ  0000000140008ebc f i MSVCRT:throw_bad_alloc.obj
 0001:00007ebc       ??1bad_array_new_length@std@@UEAA@XZ 0000000140008ebc f i MSVCRT:throw_bad_alloc.obj
 0001:00007ed0       ??_Ebad_alloc@std@@UEAAPEAXI@Z 0000000140008ed0 f i MSVCRT:throw_bad_alloc.obj
 0001:00007ed0       ??_Ebad_array_new_length@std@@UEAAPEAXI@Z 0000000140008ed0 f i MSVCRT:throw_bad_alloc.obj
 0001:00007ed0       ??_Eexception@std@@UEAAPEAXI@Z 0000000140008ed0 f i MSVCRT:throw_bad_alloc.obj
 0001:00007ed0       ??_Gbad_alloc@std@@UEAAPEAXI@Z 0000000140008ed0 f i MSVCRT:throw_bad_alloc.obj
 0001:00007ed0       ??_Gbad_array_new_length@std@@UEAAPEAXI@Z 0000000140008ed0 f i MSVCRT:throw_bad_alloc.obj
 0001:00007ed0       ??_Gexception@std@@UEAAPEAXI@Z 0000000140008ed0 f i MSVCRT:throw_bad_alloc.obj
 0001:00007f14       ?__scrt_throw_std_bad_alloc@@YAXXZ 0000000140008f14 f   MSVCRT:throw_bad_alloc.obj
 0001:00007f34       ?__scrt_throw_std_bad_array_new_length@@YAXXZ 0000000140008f34 f   MSVCRT:throw_bad_alloc.obj
 0001:00007f54       ?what@exception@std@@UEBAPEBDXZ 0000000140008f54 f i MSVCRT:throw_bad_alloc.obj
 0001:00007f68       __scrt_acquire_startup_lock 0000000140008f68 f   MSVCRT:utility.obj
 0001:00007fa4       __scrt_initialize_crt      0000000140008fa4 f   MSVCRT:utility.obj
 0001:00007ff0       __scrt_initialize_onexit_tables 0000000140008ff0 f   MSVCRT:utility.obj
 0001:0000807c       __scrt_is_nonwritable_in_current_image 000000014000907c f   MSVCRT:utility.obj
 0001:00008114       __scrt_release_startup_lock 0000000140009114 f   MSVCRT:utility.obj
 0001:00008138       __scrt_uninitialize_crt    0000000140009138 f   MSVCRT:utility.obj
 0001:00008164       _onexit                    0000000140009164 f   MSVCRT:utility.obj
 0001:000081a0       atexit                     00000001400091a0 f   MSVCRT:utility.obj
 0001:000081b8       __security_init_cookie     00000001400091b8 f   MSVCRT:gs_support.obj
 0001:00008264       __scrt_exe_initialize_mta  0000000140009264 f   MSVCRT:utility_desktop.obj
 0001:00008264       __scrt_initialize_winrt    0000000140009264 f   MSVCRT:utility_desktop.obj
 0001:00008264       __scrt_stub_for_initialize_mta 0000000140009264 f   MSVCRT:utility_desktop.obj
 0001:00008264       _get_startup_commit_mode   0000000140009264 f   MSVCRT:commit_mode.obj
 0001:00008264       _get_startup_new_mode      0000000140009264 f   MSVCRT:new_mode.obj
 0001:00008264       _get_startup_thread_locale_mode 0000000140009264 f   MSVCRT:thread_locale.obj
 0001:00008264       _matherr                   0000000140009264 f   MSVCRT:matherr.obj
 0001:00008268       _get_startup_argv_mode     0000000140009268 f   MSVCRT:argv_mode.obj
 0001:00008270       _get_startup_file_mode     0000000140009270 f   MSVCRT:file_mode.obj
 0001:00008278       ?__scrt_initialize_type_info@@YAXXZ 0000000140009278 f   MSVCRT:tncleanup.obj
 0001:00008288       __acrt_initialize          0000000140009288 f   MSVCRT:ucrt_stubs.obj
 0001:00008288       __acrt_uninitialize        0000000140009288 f   MSVCRT:ucrt_stubs.obj
 0001:00008288       __scrt_stub_for_acrt_initialize 0000000140009288 f   MSVCRT:ucrt_stubs.obj
 0001:00008288       __scrt_stub_for_acrt_uninitialize 0000000140009288 f   MSVCRT:ucrt_stubs.obj
 0001:00008288       __vcrt_initialize          0000000140009288 f   MSVCRT:ucrt_stubs.obj
 0001:00008288       __vcrt_uninitialize        0000000140009288 f   MSVCRT:ucrt_stubs.obj
 0001:00008288       _should_initialize_environment 0000000140009288 f   MSVCRT:env_mode.obj
 0001:0000828c       _guard_check_icall_nop     000000014000928c f   MSVCRT:guard_support.obj
 0001:0000828c       _initialize_denormal_control 000000014000928c f   MSVCRT:denormal_control.obj
 0001:0000828c       _initialize_invalid_parameter_handler 000000014000928c f   MSVCRT:invalid_parameter_handler.obj
 0001:00008290       __local_stdio_scanf_options 0000000140009290 f i MSVCRT:default_local_stdio_options.obj
 0001:00008298       __scrt_initialize_default_local_stdio_options 0000000140009298 f   MSVCRT:default_local_stdio_options.obj
 0001:000082b4       __scrt_is_user_matherr_present 00000001400092b4 f   MSVCRT:matherr_detection.obj
 0001:000082c0       __scrt_get_dyn_tls_init_callback 00000001400092c0 f   MSVCRT:dyn_tls_init.obj
 0001:000082c8       __scrt_get_dyn_tls_dtor_callback 00000001400092c8 f   MSVCRT:dyn_tls_dtor.obj
 0001:000082d0       __crt_debugger_hook        00000001400092d0 f   MSVCRT:utility_desktop.obj
 0001:000082d8       __scrt_fastfail            00000001400092d8 f   MSVCRT:utility_desktop.obj
 0001:00008424       __scrt_get_show_window_mode 0000000140009424 f   MSVCRT:utility_desktop.obj
 0001:00008460       __scrt_initialize_mta      0000000140009460 f   MSVCRT:utility_desktop.obj
 0001:00008468       __scrt_is_managed_app      0000000140009468 f   MSVCRT:utility_desktop.obj
 0001:000084bc       __scrt_set_unhandled_exception_filter 00000001400094bc f   MSVCRT:utility_desktop.obj
 0001:000084cc       __scrt_unhandled_exception_filter 00000001400094cc f   MSVCRT:utility_desktop.obj
 0001:00008528       _RTC_Initialize            0000000140009528 f   MSVCRT:initsect.obj
 0001:00008564       _RTC_Terminate             0000000140009564 f   MSVCRT:initsect.obj
 0001:000085a0       ??_Etype_info@@UEAAPEAXI@Z 00000001400095a0 f i MSVCRT:std_type_info_static.obj
 0001:000085a0       ??_Gtype_info@@UEAAPEAXI@Z 00000001400095a0 f i MSVCRT:std_type_info_static.obj
 0001:000085cc       __isa_available_init       00000001400095cc f   MSVCRT:cpu_disp.obj
 0001:00008778       __scrt_is_ucrt_dll_in_use  0000000140009778 f   MSVCRT:ucrt_detection.obj
 0001:00008790       memcpy                     0000000140009790 f   vcruntime:VCRUNTIME140.dll
 0001:00008796       memset                     0000000140009796 f   vcruntime:VCRUNTIME140.dll
 0001:0000879c       __CxxFrameHandler4         000000014000979c f   vcruntime:VCRUNTIME140_1.dll
 0001:000087a2       __C_specific_handler       00000001400097a2 f   vcruntime:VCRUNTIME140.dll
 0001:000087a8       __std_exception_copy       00000001400097a8 f   vcruntime:VCRUNTIME140.dll
 0001:000087ae       __std_exception_destroy    00000001400097ae f   vcruntime:VCRUNTIME140.dll
 0001:000087b4       _CxxThrowException         00000001400097b4 f   vcruntime:VCRUNTIME140.dll
 0001:000087ba       __current_exception        00000001400097ba f   vcruntime:VCRUNTIME140.dll
 0001:000087c0       __current_exception_context 00000001400097c0 f   vcruntime:VCRUNTIME140.dll
 0001:000087c6       strlen                     00000001400097c6 f   ucrt:api-ms-win-crt-string-l1-1-0.dll
 0001:000087cc       strcpy                     00000001400097cc f   ucrt:api-ms-win-crt-string-l1-1-0.dll
 0001:000087d2       strcmp                     00000001400097d2 f   ucrt:api-ms-win-crt-string-l1-1-0.dll
 0001:000087d8       _callnewh                  00000001400097d8 f   ucrt:api-ms-win-crt-heap-l1-1-0.dll
 0001:000087de       malloc                     00000001400097de f   ucrt:api-ms-win-crt-heap-l1-1-0.dll
 0001:000087e4       _seh_filter_exe            00000001400097e4 f   ucrt:api-ms-win-crt-runtime-l1-1-0.dll
 0001:000087ea       _set_app_type              00000001400097ea f   ucrt:api-ms-win-crt-runtime-l1-1-0.dll
 0001:000087f0       __setusermatherr           00000001400097f0 f   ucrt:api-ms-win-crt-math-l1-1-0.dll
 0001:000087f6       _configure_narrow_argv     00000001400097f6 f   ucrt:api-ms-win-crt-runtime-l1-1-0.dll
 0001:000087fc       _initialize_narrow_environment 00000001400097fc f   ucrt:api-ms-win-crt-runtime-l1-1-0.dll
 0001:00008802       _get_narrow_winmain_command_line 0000000140009802 f   ucrt:api-ms-win-crt-runtime-l1-1-0.dll
 0001:00008808       _initterm                  0000000140009808 f   ucrt:api-ms-win-crt-runtime-l1-1-0.dll
 0001:0000880e       _initterm_e                000000014000980e f   ucrt:api-ms-win-crt-runtime-l1-1-0.dll
 0001:00008814       exit                       0000000140009814 f   ucrt:api-ms-win-crt-runtime-l1-1-0.dll
 0001:0000881a       _exit                      000000014000981a f   ucrt:api-ms-win-crt-runtime-l1-1-0.dll
 0001:00008820       _set_fmode                 0000000140009820 f   ucrt:api-ms-win-crt-stdio-l1-1-0.dll
 0001:00008826       _cexit                     0000000140009826 f   ucrt:api-ms-win-crt-runtime-l1-1-0.dll
 0001:0000882c       _c_exit                    000000014000982c f   ucrt:api-ms-win-crt-runtime-l1-1-0.dll
 0001:00008832       _register_thread_local_exe_atexit_callback 0000000140009832 f   ucrt:api-ms-win-crt-runtime-l1-1-0.dll
 0001:00008838       _configthreadlocale        0000000140009838 f   ucrt:api-ms-win-crt-locale-l1-1-0.dll
 0001:0000883e       _set_new_mode              000000014000983e f   ucrt:api-ms-win-crt-heap-l1-1-0.dll
 0001:00008844       __p__commode               0000000140009844 f   ucrt:api-ms-win-crt-stdio-l1-1-0.dll
 0001:0000884a       free                       000000014000984a f   ucrt:api-ms-win-crt-heap-l1-1-0.dll
 0001:00008850       _initialize_onexit_table   0000000140009850 f   ucrt:api-ms-win-crt-runtime-l1-1-0.dll
 0001:00008856       _register_onexit_function  0000000140009856 f   ucrt:api-ms-win-crt-runtime-l1-1-0.dll
 0001:0000885c       _crt_atexit                000000014000985c f   ucrt:api-ms-win-crt-runtime-l1-1-0.dll
 0001:00008862       terminate                  0000000140009862 f   ucrt:api-ms-win-crt-runtime-l1-1-0.dll
 0001:00008880       _guard_dispatch_icall_nop  0000000140009880 f   MSVCRT:guard_dispatch.obj
 0001:000088a0       _guard_xfg_dispatch_icall_nop 00000001400098a0 f   MSVCRT:guard_xfg_dispatch.obj
 0002:00000000       __imp_InitCommonControlsEx 000000014000a000     comctl32:COMCTL32.dll
 0002:00000008       \177COMCTL32_NULL_THUNK_DATA 000000014000a008     comctl32:COMCTL32.dll
 0002:00000010       __imp_GetStockObject       000000014000a010     gdi32:GDI32.dll
 0002:00000018       \177GDI32_NULL_THUNK_DATA  000000014000a018     gdi32:GDI32.dll
 0002:00000020       __imp_GetModuleHandleW     000000014000a020     kernel32:KERNEL32.dll
 0002:00000028       __imp_GetStartupInfoW      000000014000a028     kernel32:KERNEL32.dll
 0002:00000030       __imp_IsDebuggerPresent    000000014000a030     kernel32:KERNEL32.dll
 0002:00000038       __imp_InitializeSListHead  000000014000a038     kernel32:KERNEL32.dll
 0002:00000040       __imp_GetCurrentThreadId   000000014000a040     kernel32:KERNEL32.dll
 0002:00000048       __imp_GetCurrentProcessId  000000014000a048     kernel32:KERNEL32.dll
 0002:00000050       __imp_QueryPerformanceCounter 000000014000a050     kernel32:KERNEL32.dll
 0002:00000058       __imp_IsProcessorFeaturePresent 000000014000a058     kernel32:KERNEL32.dll
 0002:00000060       __imp_TerminateProcess     000000014000a060     kernel32:KERNEL32.dll
 0002:00000068       __imp_GetCurrentProcess    000000014000a068     kernel32:KERNEL32.dll
 0002:00000070       __imp_SetUnhandledExceptionFilter 000000014000a070     kernel32:KERNEL32.dll
 0002:00000078       __imp_UnhandledExceptionFilter 000000014000a078     kernel32:KERNEL32.dll
 0002:00000080       __imp_RtlVirtualUnwind     000000014000a080     kernel32:KERNEL32.dll
 0002:00000088       __imp_RtlLookupFunctionEntry 000000014000a088     kernel32:KERNEL32.dll
 0002:00000090       __imp_RtlCaptureContext    000000014000a090     kernel32:KERNEL32.dll
 0002:00000098       __imp_FormatMessageA       000000014000a098     kernel32:KERNEL32.dll
 0002:000000a0       __imp_LocalFree            000000014000a0a0     kernel32:KERNEL32.dll
 0002:000000a8       __imp_GetSystemTimeAsFileTime 000000014000a0a8     kernel32:KERNEL32.dll
 0002:000000b0       __imp_LoadLibraryA         000000014000a0b0     kernel32:KERNEL32.dll
 0002:000000b8       __imp_GetProcAddress       000000014000a0b8     kernel32:KERNEL32.dll
 0002:000000c0       __imp_FreeLibrary          000000014000a0c0     kernel32:KERNEL32.dll
 0002:000000c8       __imp_GetLastError         000000014000a0c8     kernel32:KERNEL32.dll
 0002:000000d0       \177KERNEL32_NULL_THUNK_DATA 000000014000a0d0     kernel32:KERNEL32.dll
 0002:000000d8       __imp_EnumChildWindows     000000014000a0d8     user32:USER32.dll
 0002:000000e0       __imp_ScreenToClient       000000014000a0e0     user32:USER32.dll
 0002:000000e8       __imp_GetClassNameA        000000014000a0e8     user32:USER32.dll
 0002:000000f0       __imp_LoadCursorA          000000014000a0f0     user32:USER32.dll
 0002:000000f8       __imp_LoadIconA            000000014000a0f8     user32:USER32.dll
 0002:00000100       __imp_RegisterWindowMessageA 000000014000a100     user32:USER32.dll
 0002:00000108       __imp_GetCursorPos         000000014000a108     user32:USER32.dll
 0002:00000110       __imp_GetClientRect        000000014000a110     user32:USER32.dll
 0002:00000118       __imp_UpdateWindow         000000014000a118     user32:USER32.dll
 0002:00000120       __imp_TrackPopupMenu       000000014000a120     user32:USER32.dll
 0002:00000128       __imp_GetSubMenu           000000014000a128     user32:USER32.dll
 0002:00000130       __imp_LoadMenuA            000000014000a130     user32:USER32.dll
 0002:00000138       __imp_GetDlgItem           000000014000a138     user32:USER32.dll
 0002:00000140       __imp_EndDialog            000000014000a140     user32:USER32.dll
 0002:00000148       __imp_SetWindowPos         000000014000a148     user32:USER32.dll
 0002:00000150       __imp_ShowWindow           000000014000a150     user32:USER32.dll
 0002:00000158       __imp_DestroyWindow        000000014000a158     user32:USER32.dll
 0002:00000160       __imp_CreateWindowExA      000000014000a160     user32:USER32.dll
 0002:00000168       __imp_RegisterClassExA     000000014000a168     user32:USER32.dll
 0002:00000170       __imp_PostQuitMessage      000000014000a170     user32:USER32.dll
 0002:00000178       __imp_DefWindowProcA       000000014000a178     user32:USER32.dll
 0002:00000180       __imp_SendMessageA         000000014000a180     user32:USER32.dll
 0002:00000188       __imp_DispatchMessageA     000000014000a188     user32:USER32.dll
 0002:00000190       __imp_TranslateMessage     000000014000a190     user32:USER32.dll
 0002:00000198       __imp_GetMessageA          000000014000a198     user32:USER32.dll
 0002:000001a0       __imp_wsprintfA            000000014000a1a0     user32:USER32.dll
 0002:000001a8       __imp_SetDlgItemTextA      000000014000a1a8     user32:USER32.dll
 0002:000001b0       __imp_EnumWindows          000000014000a1b0     user32:USER32.dll
 0002:000001b8       \177USER32_NULL_THUNK_DATA 000000014000a1b8     user32:USER32.dll
 0002:000001c0       __imp_memcpy               000000014000a1c0     vcruntime:VCRUNTIME140.dll
 0002:000001c8       __imp_memset               000000014000a1c8     vcruntime:VCRUNTIME140.dll
 0002:000001d0       __imp___current_exception_context 000000014000a1d0     vcruntime:VCRUNTIME140.dll
 0002:000001d8       __imp___C_specific_handler 000000014000a1d8     vcruntime:VCRUNTIME140.dll
 0002:000001e0       __imp___std_exception_copy 000000014000a1e0     vcruntime:VCRUNTIME140.dll
 0002:000001e8       __imp___std_exception_destroy 000000014000a1e8     vcruntime:VCRUNTIME140.dll
 0002:000001f0       __imp__CxxThrowException   000000014000a1f0     vcruntime:VCRUNTIME140.dll
 0002:000001f8       __imp___current_exception  000000014000a1f8     vcruntime:VCRUNTIME140.dll
 0002:00000200       \177VCRUNTIME140_NULL_THUNK_DATA 000000014000a200     vcruntime:VCRUNTIME140.dll
 0002:00000208       __imp___CxxFrameHandler4   000000014000a208     vcruntime:VCRUNTIME140_1.dll
 0002:00000210       \177VCRUNTIME140_1_NULL_THUNK_DATA 000000014000a210     vcruntime:VCRUNTIME140_1.dll
 0002:00000218       __imp_getenv               000000014000a218     ucrt:api-ms-win-crt-environment-l1-1-0.dll
 0002:00000220       \177api-ms-win-crt-environment-l1-1-0_NULL_THUNK_DATA 000000014000a220     ucrt:api-ms-win-crt-environment-l1-1-0.dll
 0002:00000228       __imp_malloc               000000014000a228     ucrt:api-ms-win-crt-heap-l1-1-0.dll
 0002:00000230       __imp__callnewh            000000014000a230     ucrt:api-ms-win-crt-heap-l1-1-0.dll
 0002:00000238       __imp__set_new_mode        000000014000a238     ucrt:api-ms-win-crt-heap-l1-1-0.dll
 0002:00000240       __imp_free                 000000014000a240     ucrt:api-ms-win-crt-heap-l1-1-0.dll
 0002:00000248       \177api-ms-win-crt-heap-l1-1-0_NULL_THUNK_DATA 000000014000a248     ucrt:api-ms-win-crt-heap-l1-1-0.dll
 0002:00000250       __imp__configthreadlocale  000000014000a250     ucrt:api-ms-win-crt-locale-l1-1-0.dll
 0002:00000258       \177api-ms-win-crt-locale-l1-1-0_NULL_THUNK_DATA 000000014000a258     ucrt:api-ms-win-crt-locale-l1-1-0.dll
 0002:00000260       __imp___setusermatherr     000000014000a260     ucrt:api-ms-win-crt-math-l1-1-0.dll
 0002:00000268       \177api-ms-win-crt-math-l1-1-0_NULL_THUNK_DATA 000000014000a268     ucrt:api-ms-win-crt-math-l1-1-0.dll
 0002:00000270       __imp_terminate            000000014000a270     ucrt:api-ms-win-crt-runtime-l1-1-0.dll
 0002:00000278       __imp__crt_atexit          000000014000a278     ucrt:api-ms-win-crt-runtime-l1-1-0.dll
 0002:00000280       __imp__register_onexit_function 000000014000a280     ucrt:api-ms-win-crt-runtime-l1-1-0.dll
 0002:00000288       __imp__initialize_onexit_table 000000014000a288     ucrt:api-ms-win-crt-runtime-l1-1-0.dll
 0002:00000290       __imp__register_thread_local_exe_atexit_callback 000000014000a290     ucrt:api-ms-win-crt-runtime-l1-1-0.dll
 0002:00000298       __imp__seh_filter_exe      000000014000a298     ucrt:api-ms-win-crt-runtime-l1-1-0.dll
 0002:000002a0       __imp__set_app_type        000000014000a2a0     ucrt:api-ms-win-crt-runtime-l1-1-0.dll
 0002:000002a8       __imp__cexit               000000014000a2a8     ucrt:api-ms-win-crt-runtime-l1-1-0.dll
 0002:000002b0       __imp__configure_narrow_argv 000000014000a2b0     ucrt:api-ms-win-crt-runtime-l1-1-0.dll
 0002:000002b8       __imp__initialize_narrow_environment 000000014000a2b8     ucrt:api-ms-win-crt-runtime-l1-1-0.dll
 0002:000002c0       __imp__c_exit              000000014000a2c0     ucrt:api-ms-win-crt-runtime-l1-1-0.dll
 0002:000002c8       __imp__initterm            000000014000a2c8     ucrt:api-ms-win-crt-runtime-l1-1-0.dll
 0002:000002d0       __imp__initterm_e          000000014000a2d0     ucrt:api-ms-win-crt-runtime-l1-1-0.dll
 0002:000002d8       __imp_exit                 000000014000a2d8     ucrt:api-ms-win-crt-runtime-l1-1-0.dll
 0002:000002e0       __imp__exit                000000014000a2e0     ucrt:api-ms-win-crt-runtime-l1-1-0.dll
 0002:000002e8       __imp__get_narrow_winmain_command_line 000000014000a2e8     ucrt:api-ms-win-crt-runtime-l1-1-0.dll
 0002:000002f0       \177api-ms-win-crt-runtime-l1-1-0_NULL_THUNK_DATA 000000014000a2f0     ucrt:api-ms-win-crt-runtime-l1-1-0.dll
 0002:000002f8       __imp_fclose               000000014000a2f8     ucrt:api-ms-win-crt-stdio-l1-1-0.dll
 0002:00000300       __imp_fopen                000000014000a300     ucrt:api-ms-win-crt-stdio-l1-1-0.dll
 0002:00000308       __imp___stdio_common_vfwprintf 000000014000a308     ucrt:api-ms-win-crt-stdio-l1-1-0.dll
 0002:00000310       __imp___acrt_iob_func      000000014000a310     ucrt:api-ms-win-crt-stdio-l1-1-0.dll
 0002:00000318       __imp___p__commode         000000014000a318     ucrt:api-ms-win-crt-stdio-l1-1-0.dll
 0002:00000320       __imp___stdio_common_vsprintf 000000014000a320     ucrt:api-ms-win-crt-stdio-l1-1-0.dll
 0002:00000328       __imp___stdio_common_vfprintf 000000014000a328     ucrt:api-ms-win-crt-stdio-l1-1-0.dll
 0002:00000330       __imp__set_fmode           000000014000a330     ucrt:api-ms-win-crt-stdio-l1-1-0.dll
 0002:00000338       __imp_fflush               000000014000a338     ucrt:api-ms-win-crt-stdio-l1-1-0.dll
 0002:00000340       \177api-ms-win-crt-stdio-l1-1-0_NULL_THUNK_DATA 000000014000a340     ucrt:api-ms-win-crt-stdio-l1-1-0.dll
 0002:00000348       __imp_wcscmp               000000014000a348     ucrt:api-ms-win-crt-string-l1-1-0.dll
 0002:00000350       __imp_strncpy              000000014000a350     ucrt:api-ms-win-crt-string-l1-1-0.dll
 0002:00000358       __imp_strlen               000000014000a358     ucrt:api-ms-win-crt-string-l1-1-0.dll
 0002:00000360       __imp_strcmp               000000014000a360     ucrt:api-ms-win-crt-string-l1-1-0.dll
 0002:00000368       __imp_strcpy               000000014000a368     ucrt:api-ms-win-crt-string-l1-1-0.dll
 0002:00000370       __imp_strncat              000000014000a370     ucrt:api-ms-win-crt-string-l1-1-0.dll
 0002:00000378       \177api-ms-win-crt-string-l1-1-0_NULL_THUNK_DATA 000000014000a378     ucrt:api-ms-win-crt-string-l1-1-0.dll
 0002:00000380       __imp_asctime              000000014000a380     ucrt:api-ms-win-crt-time-l1-1-0.dll
 0002:00000388       __imp__time64              000000014000a388     ucrt:api-ms-win-crt-time-l1-1-0.dll
 0002:00000390       __imp__localtime64         000000014000a390     ucrt:api-ms-win-crt-time-l1-1-0.dll
 0002:00000398       \177api-ms-win-crt-time-l1-1-0_NULL_THUNK_DATA 000000014000a398     ucrt:api-ms-win-crt-time-l1-1-0.dll
 0002:000003a0       __guard_check_icall_fptr   000000014000a3a0     MSVCRT:guard_support.obj
 0002:000003a8       __guard_xfg_check_icall_fptr 000000014000a3a8     MSVCRT:guard_support.obj
 0002:000003b0       __guard_dispatch_icall_fptr 000000014000a3b0     MSVCRT:guard_support.obj
 0002:000003b8       __guard_xfg_dispatch_icall_fptr 000000014000a3b8     MSVCRT:guard_support.obj
 0002:000003c0       __guard_xfg_table_dispatch_icall_fptr 000000014000a3c0     MSVCRT:guard_support.obj
 0002:000003c8       __castguard_check_failure_os_handled_fptr 000000014000a3c8     MSVCRT:guard_support.obj
 0002:000003d0       __guard_memcpy_fptr        000000014000a3d0     vcruntime:softmemtag.obj
 0002:000003d8       __xc_a                     000000014000a3d8     MSVCRT:initializers.obj
 0002:000003e8       __xc_z                     000000014000a3e8     MSVCRT:initializers.obj
 0002:000003f0       __xi_a                     000000014000a3f0     MSVCRT:initializers.obj
 0002:00000408       __xi_z                     000000014000a408     MSVCRT:initializers.obj
 0002:00000410       __xp_a                     000000014000a410     MSVCRT:initializers.obj
 0002:00000418       __xp_z                     000000014000a418     MSVCRT:initializers.obj
 0002:00000420       __xt_a                     000000014000a420     MSVCRT:initializers.obj
 0002:00000428       __xt_z                     000000014000a428     MSVCRT:initializers.obj
 0002:00001ee0       ??_7exception@std@@6B@     000000014000bee0     MSVCRT:throw_bad_alloc.obj
 0002:00001ef0       ??_C@_0BC@EOODALEL@Unknown?5exception@ 000000014000bef0     MSVCRT:throw_bad_alloc.obj
 0002:00001f10       ??_7bad_alloc@std@@6B@     000000014000bf10     MSVCRT:throw_bad_alloc.obj
 0002:00001f20       ??_C@_0P@GHFPNOJB@bad?5allocation@ 000000014000bf20     MSVCRT:throw_bad_alloc.obj
 0002:00001f38       ??_7bad_array_new_length@std@@6B@ 000000014000bf38     MSVCRT:throw_bad_alloc.obj
 0002:00001f48       ??_C@_0BF@KINCDENJ@bad?5array?5new?5length@ 000000014000bf48     MSVCRT:throw_bad_alloc.obj
 0002:00001f60       __xmm@ffffffffffffffffffffffffffffffff 000000014000bf60     MSVCRT:utility.obj
 0002:00001f78       ??_7type_info@@6B@         000000014000bf78     MSVCRT:std_type_info_static.obj
 0002:00001f80       _load_config_used          000000014000bf80     MSVCRT:loadcfg.obj
 0002:00002180       ??_R4exception@std@@6B@    000000014000c180     MSVCRT:throw_bad_alloc.obj
 0002:000021a8       ??_R3exception@std@@8      000000014000c1a8     MSVCRT:throw_bad_alloc.obj
 0002:000021c0       ??_R2exception@std@@8      000000014000c1c0     MSVCRT:throw_bad_alloc.obj
 0002:000021d0       ??_R1A@?0A@EA@exception@std@@8 000000014000c1d0     MSVCRT:throw_bad_alloc.obj
 0002:000021f8       ??_R4bad_alloc@std@@6B@    000000014000c1f8     MSVCRT:throw_bad_alloc.obj
 0002:00002220       ??_R3bad_alloc@std@@8      000000014000c220     MSVCRT:throw_bad_alloc.obj
 0002:00002238       ??_R2bad_alloc@std@@8      000000014000c238     MSVCRT:throw_bad_alloc.obj
 0002:00002250       ??_R1A@?0A@EA@bad_alloc@std@@8 000000014000c250     MSVCRT:throw_bad_alloc.obj
 0002:00002278       ??_R4bad_array_new_length@std@@6B@ 000000014000c278     MSVCRT:throw_bad_alloc.obj
 0002:000022a0       ??_R3bad_array_new_length@std@@8 000000014000c2a0     MSVCRT:throw_bad_alloc.obj
 0002:000022b8       ??_R2bad_array_new_length@std@@8 000000014000c2b8     MSVCRT:throw_bad_alloc.obj
 0002:000022d8       ??_R1A@?0A@EA@bad_array_new_length@std@@8 000000014000c2d8     MSVCRT:throw_bad_alloc.obj
 0002:00002300       ??_R4type_info@@6B@        000000014000c300     MSVCRT:std_type_info_static.obj
 0002:00002328       ??_R3type_info@@8          000000014000c328     MSVCRT:std_type_info_static.obj
 0002:00002340       ??_R2type_info@@8          000000014000c340     MSVCRT:std_type_info_static.obj
 0002:00002350       ??_R1A@?0A@EA@type_info@@8 000000014000c350     MSVCRT:std_type_info_static.obj
 0002:00002374       __volatile_metadata        000000014000c374     <linker-defined>
 0002:00002760       __rtc_iaa                  000000014000c760     MSVCRT:initsect.obj
 0002:00002768       __rtc_izz                  000000014000c768     MSVCRT:initsect.obj
 0002:00002770       __rtc_taa                  000000014000c770     MSVCRT:initsect.obj
 0002:00002778       __rtc_tzz                  000000014000c778     MSVCRT:initsect.obj
 0002:00002d40       _TI2?AVbad_alloc@std@@     000000014000cd40     MSVCRT:throw_bad_alloc.obj
 0002:00002d60       _CTA2?AVbad_alloc@std@@    000000014000cd60     MSVCRT:throw_bad_alloc.obj
 0002:00002d78       _CT??_R0?AVbad_alloc@std@@@8??0bad_alloc@std@@QEAA@AEBV01@@Z24 000000014000cd78     MSVCRT:throw_bad_alloc.obj
 0002:00002da0       _CT??_R0?AVexception@std@@@8??0exception@std@@QEAA@AEBV01@@Z24 000000014000cda0     MSVCRT:throw_bad_alloc.obj
 0002:00002dc8       _TI3?AVbad_array_new_length@std@@ 000000014000cdc8     MSVCRT:throw_bad_alloc.obj
 0002:00002de8       _CTA3?AVbad_array_new_length@std@@ 000000014000cde8     MSVCRT:throw_bad_alloc.obj
 0002:00002e08       _CT??_R0?AVbad_array_new_length@std@@@8??0bad_array_new_length@std@@QEAA@AEBV01@@Z24 000000014000ce08     MSVCRT:throw_bad_alloc.obj
 0002:00002e2c       __IMPORT_DESCRIPTOR_COMCTL32 000000014000ce2c     comctl32:COMCTL32.dll
 0002:00002e40       __IMPORT_DESCRIPTOR_GDI32  000000014000ce40     gdi32:GDI32.dll
 0002:00002e54       __IMPORT_DESCRIPTOR_USER32 000000014000ce54     user32:USER32.dll
 0002:00002e68       __IMPORT_DESCRIPTOR_KERNEL32 000000014000ce68     kernel32:KERNEL32.dll
 0002:00002e7c       __IMPORT_DESCRIPTOR_VCRUNTIME140 000000014000ce7c     vcruntime:VCRUNTIME140.dll
 0002:00002e90       __IMPORT_DESCRIPTOR_VCRUNTIME140_1 000000014000ce90     vcruntime:VCRUNTIME140_1.dll
 0002:00002ea4       __IMPORT_DESCRIPTOR_api-ms-win-crt-string-l1-1-0 000000014000cea4     ucrt:api-ms-win-crt-string-l1-1-0.dll
 0002:00002eb8       __IMPORT_DESCRIPTOR_api-ms-win-crt-stdio-l1-1-0 000000014000ceb8     ucrt:api-ms-win-crt-stdio-l1-1-0.dll
 0002:00002ecc       __IMPORT_DESCRIPTOR_api-ms-win-crt-environment-l1-1-0 000000014000cecc     ucrt:api-ms-win-crt-environment-l1-1-0.dll
 0002:00002ee0       __IMPORT_DESCRIPTOR_api-ms-win-crt-time-l1-1-0 000000014000cee0     ucrt:api-ms-win-crt-time-l1-1-0.dll
 0002:00002ef4       __IMPORT_DESCRIPTOR_api-ms-win-crt-heap-l1-1-0 000000014000cef4     ucrt:api-ms-win-crt-heap-l1-1-0.dll
 0002:00002f08       __IMPORT_DESCRIPTOR_api-ms-win-crt-runtime-l1-1-0 000000014000cf08     ucrt:api-ms-win-crt-runtime-l1-1-0.dll
 0002:00002f1c       __IMPORT_DESCRIPTOR_api-ms-win-crt-math-l1-1-0 000000014000cf1c     ucrt:api-ms-win-crt-math-l1-1-0.dll
 0002:00002f30       __IMPORT_DESCRIPTOR_api-ms-win-crt-locale-l1-1-0 000000014000cf30     ucrt:api-ms-win-crt-locale-l1-1-0.dll
 0002:00002f44       __NULL_IMPORT_DESCRIPTOR   000000014000cf44     comctl32:COMCTL32.dll
 0003:00000b30       ?depth@@3HA                000000014000eb30     jaccesswalker.obj
 0003:00000b38       ?theJaccesswalkerClassName@@3PADA 000000014000eb38     jaccesswalker.obj
 0003:00000b50       ?theAccessInfoClassName@@3PADA 000000014000eb50     jaccesswalker.obj
 0003:00000b90       __security_cookie_complement 000000014000eb90     MSVCRT:gs_cookie.obj
 0003:00000b98       __security_cookie          000000014000eb98     MSVCRT:gs_cookie.obj
 0003:00000ba0       _fltused                   000000014000eba0     MSVCRT:fltused.obj
 0003:00000ba4       __scrt_native_dllmain_reason 000000014000eba4     MSVCRT:utility.obj
 0003:00000ba8       __scrt_default_matherr     000000014000eba8     MSVCRT:matherr.obj
 0003:00000bb0       __isa_available            000000014000ebb0     MSVCRT:cpu_disp.obj
 0003:00000bb4       __isa_enabled              000000014000ebb4     MSVCRT:cpu_disp.obj
 0003:00000bb8       __memset_fast_string_threshold 000000014000ebb8     MSVCRT:cpu_disp.obj
 0003:00000bc0       __memset_nt_threshold      000000014000ebc0     MSVCRT:cpu_disp.obj
 0003:00000bd0       __scrt_ucrt_dll_is_in_use  000000014000ebd0     MSVCRT:ucrt_stubs.obj
 0003:00000bd8       ??_R0?AVbad_alloc@std@@@8  000000014000ebd8     MSVCRT:throw_bad_alloc.obj
 0003:00000c00       ??_R0?AVexception@std@@@8  000000014000ec00     MSVCRT:throw_bad_alloc.obj
 0003:00000c28       ??_R0?AVbad_array_new_length@std@@@8 000000014000ec28     MSVCRT:throw_bad_alloc.obj
 0003:00000c58       ??_R0?AVtype_info@@@8      000000014000ec58     MSVCRT:std_type_info_static.obj
 0003:00000c80       theAccessBridgeInitializedFlag 000000014000ec80     AccessBridgeCalls.obj
 0003:00000c88       ?_OptionsStorage@?1??__local_stdio_printf_options@@9@4_KA 000000014000ec88     AccessBridgeDebug.obj
 0003:00000da0       ?theFromJavaHelloMsgID@@3IA 000000014000eda0     AccessBridgeMessages.obj
 0003:00000da4       ?theFromWindowsHelloMsgID@@3IA 000000014000eda4     AccessBridgeMessages.obj
 0003:00000da8       ?g_LogStringCallback@@3P6AXPEBD@ZEA 000000014000eda8     AccessInfo.obj
 0003:00000df0       ?ourHwnd@@3PEAUHWND__@@EA  000000014000edf0     jaccesswalker.obj
 0003:00000df8       ?topLevelWindow@@3PEAUHWND__@@EA 000000014000edf8     jaccesswalker.obj
 0003:00000e00       ?logfile@@3PEAU_iobuf@@EA  000000014000ee00     jaccesswalker.obj
 0003:00000e08       ?popupMenu@@3PEAUHMENU__@@EA 000000014000ee08     jaccesswalker.obj
 0003:00000e10       ?theJaccesswalkerWindow@@3PEAUHWND__@@EA 000000014000ee10     jaccesswalker.obj
 0003:00000e18       ?theTreeControlWindow@@3PEAUHWND__@@EA 000000014000ee18     jaccesswalker.obj
 0003:00000e20       ?theInstance@@3PEAUHINSTANCE__@@EA 000000014000ee20     jaccesswalker.obj
 0003:00000e28       ?theJaccesswalker@@3PEAVJaccesswalker@@EA 000000014000ee28     jaccesswalker.obj
 0003:00000e30       ?theSelectedNode@@3PEAVAccessibleNode@@EA 000000014000ee30     jaccesswalker.obj
 0003:00000e38       ?thePopupNode@@3PEAVAccessibleNode@@EA 000000014000ee38     jaccesswalker.obj
 0003:00000e40       ?theSelectedAccessibleContext@@3_JA 000000014000ee40     jaccesswalker.obj
 0003:00000e48       ?hwndTV@@3PEAUHWND__@@EA   000000014000ee48     jaccesswalker.obj
 0003:000013c0       __scrt_current_native_startup_state 000000014000f3c0     MSVCRT:utility.obj
 0003:000013c8       __scrt_native_startup_lock 000000014000f3c8     MSVCRT:utility.obj
 0003:00001410       ?__type_info_root_node@@3U__type_info_node@@A 000000014000f410     MSVCRT:tncleanup.obj
 0003:00001420       ?_OptionsStorage@?1??__local_stdio_scanf_options@@9@4_KA 000000014000f420     MSVCRT:default_local_stdio_options.obj
 0003:00001428       __scrt_debugger_hook_flag  000000014000f428     MSVCRT:utility_desktop.obj
 0003:0000142c       __favor                    000000014000f42c     MSVCRT:cpu_disp.obj
 0003:00001440       theAccessBridge            000000014000f440     <common>
 0003:00001748       theAccessBridgeInstance    000000014000f748     <common>
 0003:00001750       __dyn_tls_dtor_callback    000000014000f750     <common>
 0003:00001758       __dyn_tls_init_callback    000000014000f758     <common>

 entry point at        0001:00007db4

 Static symbols

 0000:fffed000       .debug$S                   0000000140000000     vcruntime:VCRUNTIME140.dll
 0000:fffed000       .debug$S                   0000000140000000     vcruntime:VCRUNTIME140.dll
 0000:fffed000       .debug$S                   0000000140000000     vcruntime:VCRUNTIME140.dll
 0000:fffed000       .debug$S                   0000000140000000     vcruntime:VCRUNTIME140.dll
 0000:fffed000       .debug$S                   0000000140000000     vcruntime:VCRUNTIME140.dll
 0000:fffed000       .debug$S                   0000000140000000     vcruntime:VCRUNTIME140.dll
 0000:fffed000       .debug$S                   0000000140000000     vcruntime:VCRUNTIME140.dll
 0000:fffed000       .debug$S                   0000000140000000     vcruntime:VCRUNTIME140.dll
 0000:fffed000       .debug$S                   0000000140000000     vcruntime:VCRUNTIME140.dll
 0000:fffed000       .debug$S                   0000000140000000     vcruntime:VCRUNTIME140_1.dll
 0000:fffed000       .debug$S                   0000000140000000     ucrt:api-ms-win-crt-environment-l1-1-0.dll
 0000:fffed000       .debug$S                   0000000140000000     ucrt:api-ms-win-crt-heap-l1-1-0.dll
 0000:fffed000       .debug$S                   0000000140000000     ucrt:api-ms-win-crt-heap-l1-1-0.dll
 0000:fffed000       .debug$S                   0000000140000000     ucrt:api-ms-win-crt-heap-l1-1-0.dll
 0000:fffed000       .debug$S                   0000000140000000     ucrt:api-ms-win-crt-heap-l1-1-0.dll
 0000:fffed000       .debug$S                   0000000140000000     ucrt:api-ms-win-crt-locale-l1-1-0.dll
 0000:fffed000       .debug$S                   0000000140000000     ucrt:api-ms-win-crt-math-l1-1-0.dll
 0000:fffed000       .debug$S                   0000000140000000     ucrt:api-ms-win-crt-runtime-l1-1-0.dll
 0000:fffed000       .debug$S                   0000000140000000     ucrt:api-ms-win-crt-runtime-l1-1-0.dll
 0000:fffed000       .debug$S                   0000000140000000     ucrt:api-ms-win-crt-runtime-l1-1-0.dll
 0000:fffed000       .debug$S                   0000000140000000     ucrt:api-ms-win-crt-runtime-l1-1-0.dll
 0000:fffed000       .debug$S                   0000000140000000     ucrt:api-ms-win-crt-runtime-l1-1-0.dll
 0000:fffed000       .debug$S                   0000000140000000     ucrt:api-ms-win-crt-runtime-l1-1-0.dll
 0000:fffed000       .debug$S                   0000000140000000     ucrt:api-ms-win-crt-runtime-l1-1-0.dll
 0000:fffed000       .debug$S                   0000000140000000     ucrt:api-ms-win-crt-runtime-l1-1-0.dll
 0000:fffed000       .debug$S                   0000000140000000     ucrt:api-ms-win-crt-runtime-l1-1-0.dll
 0000:fffed000       .debug$S                   0000000140000000     ucrt:api-ms-win-crt-runtime-l1-1-0.dll
 0000:fffed000       .debug$S                   0000000140000000     ucrt:api-ms-win-crt-runtime-l1-1-0.dll
 0000:fffed000       .debug$S                   0000000140000000     ucrt:api-ms-win-crt-runtime-l1-1-0.dll
 0000:fffed000       .debug$S                   0000000140000000     ucrt:api-ms-win-crt-runtime-l1-1-0.dll
 0000:fffed000       .debug$S                   0000000140000000     ucrt:api-ms-win-crt-runtime-l1-1-0.dll
 0000:fffed000       .debug$S                   0000000140000000     ucrt:api-ms-win-crt-runtime-l1-1-0.dll
 0000:fffed000       .debug$S                   0000000140000000     ucrt:api-ms-win-crt-runtime-l1-1-0.dll
 0000:fffed000       .debug$S                   0000000140000000     ucrt:api-ms-win-crt-runtime-l1-1-0.dll
 0000:fffed000       .debug$S                   0000000140000000     ucrt:api-ms-win-crt-runtime-l1-1-0.dll
 0000:fffed000       .debug$S                   0000000140000000     ucrt:api-ms-win-crt-runtime-l1-1-0.dll
 0000:fffed000       .debug$S                   0000000140000000     ucrt:api-ms-win-crt-stdio-l1-1-0.dll
 0000:fffed000       .debug$S                   0000000140000000     ucrt:api-ms-win-crt-stdio-l1-1-0.dll
 0000:fffed000       .debug$S                   0000000140000000     ucrt:api-ms-win-crt-stdio-l1-1-0.dll
 0000:fffed000       .debug$S                   0000000140000000     ucrt:api-ms-win-crt-stdio-l1-1-0.dll
 0000:fffed000       .debug$S                   0000000140000000     ucrt:api-ms-win-crt-stdio-l1-1-0.dll
 0000:fffed000       .debug$S                   0000000140000000     ucrt:api-ms-win-crt-stdio-l1-1-0.dll
 0000:fffed000       .debug$S                   0000000140000000     ucrt:api-ms-win-crt-stdio-l1-1-0.dll
 0000:fffed000       .debug$S                   0000000140000000     ucrt:api-ms-win-crt-stdio-l1-1-0.dll
 0000:fffed000       .debug$S                   0000000140000000     ucrt:api-ms-win-crt-stdio-l1-1-0.dll
 0000:fffed000       .debug$S                   0000000140000000     ucrt:api-ms-win-crt-string-l1-1-0.dll
 0000:fffed000       .debug$S                   0000000140000000     ucrt:api-ms-win-crt-string-l1-1-0.dll
 0000:fffed000       .debug$S                   0000000140000000     ucrt:api-ms-win-crt-string-l1-1-0.dll
 0000:fffed000       .debug$S                   0000000140000000     ucrt:api-ms-win-crt-string-l1-1-0.dll
 0000:fffed000       .debug$S                   0000000140000000     ucrt:api-ms-win-crt-string-l1-1-0.dll
 0000:fffed000       .debug$S                   0000000140000000     ucrt:api-ms-win-crt-string-l1-1-0.dll
 0000:fffed000       .debug$S                   0000000140000000     ucrt:api-ms-win-crt-time-l1-1-0.dll
 0000:fffed000       .debug$S                   0000000140000000     ucrt:api-ms-win-crt-time-l1-1-0.dll
 0000:fffed000       .debug$S                   0000000140000000     ucrt:api-ms-win-crt-time-l1-1-0.dll
 0000:fffed000       .debug$S                   0000000140000000     comctl32:COMCTL32.dll
 0000:fffed000       .debug$S                   0000000140000000     gdi32:GDI32.dll
 0000:fffed000       .debug$S                   0000000140000000     kernel32:KERNEL32.dll
 0000:fffed000       .debug$S                   0000000140000000     kernel32:KERNEL32.dll
 0000:fffed000       .debug$S                   0000000140000000     kernel32:KERNEL32.dll
 0000:fffed000       .debug$S                   0000000140000000     kernel32:KERNEL32.dll
 0000:fffed000       .debug$S                   0000000140000000     kernel32:KERNEL32.dll
 0000:fffed000       .debug$S                   0000000140000000     kernel32:KERNEL32.dll
 0000:fffed000       .debug$S                   0000000140000000     kernel32:KERNEL32.dll
 0000:fffed000       .debug$S                   0000000140000000     kernel32:KERNEL32.dll
 0000:fffed000       .debug$S                   0000000140000000     kernel32:KERNEL32.dll
 0000:fffed000       .debug$S                   0000000140000000     kernel32:KERNEL32.dll
 0000:fffed000       .debug$S                   0000000140000000     kernel32:KERNEL32.dll
 0000:fffed000       .debug$S                   0000000140000000     kernel32:KERNEL32.dll
 0000:fffed000       .debug$S                   0000000140000000     kernel32:KERNEL32.dll
 0000:fffed000       .debug$S                   0000000140000000     kernel32:KERNEL32.dll
 0000:fffed000       .debug$S                   0000000140000000     kernel32:KERNEL32.dll
 0000:fffed000       .debug$S                   0000000140000000     kernel32:KERNEL32.dll
 0000:fffed000       .debug$S                   0000000140000000     kernel32:KERNEL32.dll
 0000:fffed000       .debug$S                   0000000140000000     kernel32:KERNEL32.dll
 0000:fffed000       .debug$S                   0000000140000000     kernel32:KERNEL32.dll
 0000:fffed000       .debug$S                   0000000140000000     kernel32:KERNEL32.dll
 0000:fffed000       .debug$S                   0000000140000000     kernel32:KERNEL32.dll
 0000:fffed000       .debug$S                   0000000140000000     kernel32:KERNEL32.dll
 0000:fffed000       .debug$S                   0000000140000000     user32:USER32.dll
 0000:fffed000       .debug$S                   0000000140000000     user32:USER32.dll
 0000:fffed000       .debug$S                   0000000140000000     user32:USER32.dll
 0000:fffed000       .debug$S                   0000000140000000     user32:USER32.dll
 0000:fffed000       .debug$S                   0000000140000000     user32:USER32.dll
 0000:fffed000       .debug$S                   0000000140000000     user32:USER32.dll
 0000:fffed000       .debug$S                   0000000140000000     user32:USER32.dll
 0000:fffed000       .debug$S                   0000000140000000     user32:USER32.dll
 0000:fffed000       .debug$S                   0000000140000000     user32:USER32.dll
 0000:fffed000       .debug$S                   0000000140000000     user32:USER32.dll
 0000:fffed000       .debug$S                   0000000140000000     user32:USER32.dll
 0000:fffed000       .debug$S                   0000000140000000     user32:USER32.dll
 0000:fffed000       .debug$S                   0000000140000000     user32:USER32.dll
 0000:fffed000       .debug$S                   0000000140000000     user32:USER32.dll
 0000:fffed000       .debug$S                   0000000140000000     user32:USER32.dll
 0000:fffed000       .debug$S                   0000000140000000     user32:USER32.dll
 0000:fffed000       .debug$S                   0000000140000000     user32:USER32.dll
 0000:fffed000       .debug$S                   0000000140000000     user32:USER32.dll
 0000:fffed000       .debug$S                   0000000140000000     user32:USER32.dll
 0000:fffed000       .debug$S                   0000000140000000     user32:USER32.dll
 0000:fffed000       .debug$S                   0000000140000000     user32:USER32.dll
 0000:fffed000       .debug$S                   0000000140000000     user32:USER32.dll
 0000:fffed000       .debug$S                   0000000140000000     user32:USER32.dll
 0000:fffed000       .debug$S                   0000000140000000     user32:USER32.dll
 0000:fffed000       .debug$S                   0000000140000000     user32:USER32.dll
 0000:fffed000       .debug$S                   0000000140000000     user32:USER32.dll
 0000:fffed000       .debug$S                   0000000140000000     user32:USER32.dll
 0000:fffed000       .debug$S                   0000000140000000     user32:USER32.dll
 0001:00005d20       localtime                  0000000140006d20 f   AccessInfo.obj
 0001:00005d40       time                       0000000140006d40 f   AccessInfo.obj
 0001:000078a4       capture_current_context    00000001400088a4 f   MSVCRT:gs_report.obj
 0001:00007914       capture_previous_context   0000000140008914 f   MSVCRT:gs_report.obj
 0001:00007a10       $$000000                   0000000140008a10     MSVCRT:chkstk.obj
 0001:00007a70       $$000000                   0000000140008a70     MSVCRT:amdsecgs.obj
 0001:00007b5c       ?pre_c_initialization@@YAHXZ 0000000140008b5c f   MSVCRT:exe_winmain.obj
 0001:00007c14       ?post_pgo_initialization@@YAHXZ 0000000140008c14 f   MSVCRT:exe_winmain.obj
 0001:00007c24       ?pre_cpp_initialization@@YAXXZ 0000000140008c24 f   MSVCRT:exe_winmain.obj
 0001:00007c40       ?__scrt_common_main_seh@@YAHXZ 0000000140008c40 f   MSVCRT:exe_winmain.obj
 0001:00008870       $$000000                   0000000140009870     MSVCRT:guard_dispatch.obj
 0001:00008890       $$000000                   0000000140009890     MSVCRT:guard_xfg_dispatch.obj
 0001:000088b0       ?dtor$0@?0??addComponentNodes@Jaccesswalker@@QEAAXJ_JPEAVAccessibleNode@@PEAUHWND__@@PEAU_TREEITEM@@2@Z@4HA 00000001400098b0 f   jaccesswalker.obj
 0001:000088cd       ?filt$0@?0??__scrt_common_main_seh@@YAHXZ@4HA 00000001400098cd f   MSVCRT:exe_winmain.obj
 0001:000088eb       __scrt_is_nonwritable_in_current_image$filt$0 00000001400098eb f   MSVCRT:utility.obj
 0002:000003e0       ?pre_cpp_initializer@@3P6AXXZEA 000000014000a3e0     MSVCRT:exe_winmain.obj
 0002:000003f8       ?pre_c_initializer@@3P6AHXZEA 000000014000a3f8     MSVCRT:exe_winmain.obj
 0002:00000400       ?post_pgo_initializer@@3P6AHXZEA 000000014000a400     MSVCRT:exe_winmain.obj
 0002:00000430       $SG42737                   000000014000a430     AccessBridgeDebug.obj
 0002:0000044c       $SG42739                   000000014000a44c     AccessBridgeDebug.obj
 0002:00000454       $SG42740                   000000014000a454     AccessBridgeDebug.obj
 0002:00000458       $SG42742                   000000014000a458     AccessBridgeDebug.obj
 0002:00000460       $SG42743                   000000014000a460     AccessBridgeDebug.obj
 0002:00000478       $SG42770                   000000014000a478     AccessBridgeDebug.obj
 0002:00000498       $SG42771                   000000014000a498     AccessBridgeDebug.obj
 0002:000004a4       $SG42773                   000000014000a4a4     AccessBridgeDebug.obj
 0002:000004a8       $SG42784                   000000014000a4a8     AccessBridgeDebug.obj
 0002:000004b0       $SG42785                   000000014000a4b0     AccessBridgeDebug.obj
 0002:000004b8       $SG42796                   000000014000a4b8     AccessBridgeDebug.obj
 0002:000004c0       $SG42797                   000000014000a4c0     AccessBridgeDebug.obj
 0002:000004c8       $SG42808                   000000014000a4c8     AccessBridgeDebug.obj
 0002:000004d0       $SG42809                   000000014000a4d0     AccessBridgeDebug.obj
 0002:000004d8       $SG42820                   000000014000a4d8     AccessBridgeDebug.obj
 0002:000004e0       $SG42821                   000000014000a4e0     AccessBridgeDebug.obj
 0002:000004e8       $SG38103                   000000014000a4e8     AccessBridgeMessages.obj
 0002:00000508       $SG38104                   000000014000a508     AccessBridgeMessages.obj
 0002:00000530       $SG46955                   000000014000a530     AccessInfo.obj
 0002:00000534       $SG46957                   000000014000a534     AccessInfo.obj
 0002:00000538       $SG46960                   000000014000a538     AccessInfo.obj
 0002:00000548       $SG47000                   000000014000a548     AccessInfo.obj
 0002:00000574       $SG47001                   000000014000a574     AccessInfo.obj
 0002:00000578       $SG47002                   000000014000a578     AccessInfo.obj
 0002:0000057c       $SG47015                   000000014000a57c     AccessInfo.obj
 0002:00000580       $SG47157                   000000014000a580     AccessInfo.obj
 0002:000005a8       $SG47158                   000000014000a5a8     AccessInfo.obj
 0002:000005c0       $SG47159                   000000014000a5c0     AccessInfo.obj
 0002:000005e8       $SG47160                   000000014000a5e8     AccessInfo.obj
 0002:00000618       $SG47161                   000000014000a618     AccessInfo.obj
 0002:00000648       $SG47162                   000000014000a648     AccessInfo.obj
 0002:00000678       $SG47166                   000000014000a678     AccessInfo.obj
 0002:000006a8       $SG47167                   000000014000a6a8     AccessInfo.obj
 0002:000006d0       $SG47170                   000000014000a6d0     AccessInfo.obj
 0002:000006ec       $SG47171                   000000014000a6ec     AccessInfo.obj
 0002:000006f0       $SG47172                   000000014000a6f0     AccessInfo.obj
 0002:00000708       $SG47175                   000000014000a708     AccessInfo.obj
 0002:00000730       $SG47176                   000000014000a730     AccessInfo.obj
 0002:00000750       $SG47177                   000000014000a750     AccessInfo.obj
 0002:00000768       $SG47178                   000000014000a768     AccessInfo.obj
 0002:00000780       $SG47179                   000000014000a780     AccessInfo.obj
 0002:000007a8       $SG47180                   000000014000a7a8     AccessInfo.obj
 0002:000007c0       $SG47181                   000000014000a7c0     AccessInfo.obj
 0002:000007e8       $SG47182                   000000014000a7e8     AccessInfo.obj
 0002:00000808       $SG47183                   000000014000a808     AccessInfo.obj
 0002:00000828       $SG47184                   000000014000a828     AccessInfo.obj
 0002:00000858       $SG47187                   000000014000a858     AccessInfo.obj
 0002:00000880       $SG47190                   000000014000a880     AccessInfo.obj
 0002:000008c0       $SG47193                   000000014000a8c0     AccessInfo.obj
 0002:000008e8       $SG47194                   000000014000a8e8     AccessInfo.obj
 0002:00000910       $SG47195                   000000014000a910     AccessInfo.obj
 0002:00000938       $SG47198                   000000014000a938     AccessInfo.obj
 0002:00000948       $SG47201                   000000014000a948     AccessInfo.obj
 0002:00000980       $SG47202                   000000014000a980     AccessInfo.obj
 0002:00000998       $SG47205                   000000014000a998     AccessInfo.obj
 0002:000009c0       $SG47206                   000000014000a9c0     AccessInfo.obj
 0002:000009e0       $SG47207                   000000014000a9e0     AccessInfo.obj
 0002:000009f8       $SG47210                   000000014000a9f8     AccessInfo.obj
 0002:00000a20       $SG47211                   000000014000aa20     AccessInfo.obj
 0002:00000a48       $SG47215                   000000014000aa48     AccessInfo.obj
 0002:00000a70       $SG47219                   000000014000aa70     AccessInfo.obj
 0002:00000a98       $SG47220                   000000014000aa98     AccessInfo.obj
 0002:00000ab8       $SG47221                   000000014000aab8     AccessInfo.obj
 0002:00000ad8       $SG47223                   000000014000aad8     AccessInfo.obj
 0002:00000b00       $SG47225                   000000014000ab00     AccessInfo.obj
 0002:00000b20       $SG47228                   000000014000ab20     AccessInfo.obj
 0002:00000b68       $SG47231                   000000014000ab68     AccessInfo.obj
 0002:00000ba8       $SG47234                   000000014000aba8     AccessInfo.obj
 0002:00000bd0       $SG47235                   000000014000abd0     AccessInfo.obj
 0002:00000bf0       $SG47236                   000000014000abf0     AccessInfo.obj
 0002:00000c10       $SG47237                   000000014000ac10     AccessInfo.obj
 0002:00000c40       $SG47239                   000000014000ac40     AccessInfo.obj
 0002:00000c60       $SG47240                   000000014000ac60     AccessInfo.obj
 0002:00000c88       $SG47241                   000000014000ac88     AccessInfo.obj
 0002:00000cb0       $SG47242                   000000014000acb0     AccessInfo.obj
 0002:00000cd8       $SG47244                   000000014000acd8     AccessInfo.obj
 0002:00000cf8       $SG47245                   000000014000acf8     AccessInfo.obj
 0002:00000d18       $SG47246                   000000014000ad18     AccessInfo.obj
 0002:00000d38       $SG47247                   000000014000ad38     AccessInfo.obj
 0002:00000d58       $SG47248                   000000014000ad58     AccessInfo.obj
 0002:00000d70       $SG47250                   000000014000ad70     AccessInfo.obj
 0002:00000d90       $SG47251                   000000014000ad90     AccessInfo.obj
 0002:00000db0       $SG47252                   000000014000adb0     AccessInfo.obj
 0002:00000dd0       $SG47255                   000000014000add0     AccessInfo.obj
 0002:00000df8       $SG47257                   000000014000adf8     AccessInfo.obj
 0002:00000e20       $SG47258                   000000014000ae20     AccessInfo.obj
 0002:00000e40       $SG47259                   000000014000ae40     AccessInfo.obj
 0002:00000e60       $SG47260                   000000014000ae60     AccessInfo.obj
 0002:00000e88       $SG47263                   000000014000ae88     AccessInfo.obj
 0002:00000eb8       $SG47266                   000000014000aeb8     AccessInfo.obj
 0002:00000ee0       $SG47267                   000000014000aee0     AccessInfo.obj
 0002:00000f00       $SG47268                   000000014000af00     AccessInfo.obj
 0002:00000f20       $SG47270                   000000014000af20     AccessInfo.obj
 0002:00000f48       $SG47272                   000000014000af48     AccessInfo.obj
 0002:00000f68       $SG47274                   000000014000af68     AccessInfo.obj
 0002:00000f88       $SG47276                   000000014000af88     AccessInfo.obj
 0002:00000fa8       $SG47280                   000000014000afa8     AccessInfo.obj
 0002:00000fd0       $SG47281                   000000014000afd0     AccessInfo.obj
 0002:00000ff0       $SG47282                   000000014000aff0     AccessInfo.obj
 0002:00001018       $SG47283                   000000014000b018     AccessInfo.obj
 0002:00001040       $SG47284                   000000014000b040     AccessInfo.obj
 0002:00001068       $SG47285                   000000014000b068     AccessInfo.obj
 0002:00001088       $SG47286                   000000014000b088     AccessInfo.obj
 0002:000010a8       $SG47289                   000000014000b0a8     AccessInfo.obj
 0002:000010d8       $SG47290                   000000014000b0d8     AccessInfo.obj
 0002:00001108       $SG47291                   000000014000b108     AccessInfo.obj
 0002:00001120       $SG47292                   000000014000b120     AccessInfo.obj
 0002:00001138       $SG47293                   000000014000b138     AccessInfo.obj
 0002:00001158       $SG47294                   000000014000b158     AccessInfo.obj
 0002:00001170       $SG47297                   000000014000b170     AccessInfo.obj
 0002:000011b8       $SG47300                   000000014000b1b8     AccessInfo.obj
 0002:000011e0       $SG47301                   000000014000b1e0     AccessInfo.obj
 0002:000011f8       $SG47302                   000000014000b1f8     AccessInfo.obj
 0002:00001210       $SG47305                   000000014000b210     AccessInfo.obj
 0002:00001240       $SG47306                   000000014000b240     AccessInfo.obj
 0002:00001268       $SG47307                   000000014000b268     AccessInfo.obj
 0002:00001290       $SG47308                   000000014000b290     AccessInfo.obj
 0002:000012b8       $SG47309                   000000014000b2b8     AccessInfo.obj
 0002:000012d8       $SG47312                   000000014000b2d8     AccessInfo.obj
 0002:00001310       $SG47313                   000000014000b310     AccessInfo.obj
 0002:00001328       $SG47314                   000000014000b328     AccessInfo.obj
 0002:00001330       $SG47317                   000000014000b330     AccessInfo.obj
 0002:00001360       $SG47318                   000000014000b360     AccessInfo.obj
 0002:00001388       $SG47319                   000000014000b388     AccessInfo.obj
 0002:000013a0       $SG47320                   000000014000b3a0     AccessInfo.obj
 0002:000013b8       $SG47321                   000000014000b3b8     AccessInfo.obj
 0002:000013d8       $SG47322                   000000014000b3d8     AccessInfo.obj
 0002:000013f0       $SG47325                   000000014000b3f0     AccessInfo.obj
 0002:00001420       $SG47328                   000000014000b420     AccessInfo.obj
 0002:00001448       $SG47329                   000000014000b448     AccessInfo.obj
 0002:00001460       $SG47330                   000000014000b460     AccessInfo.obj
 0002:00001478       $SG47332                   000000014000b478     AccessInfo.obj
 0002:000014a0       $SG47334                   000000014000b4a0     AccessInfo.obj
 0002:000014c8       $SG47335                   000000014000b4c8     AccessInfo.obj
 0002:000014e8       $SG47336                   000000014000b4e8     AccessInfo.obj
 0002:00001500       $SG47338                   000000014000b500     AccessInfo.obj
 0002:00001528       $SG47339                   000000014000b528     AccessInfo.obj
 0002:00001548       $SG47340                   000000014000b548     AccessInfo.obj
 0002:00001568       $SG47341                   000000014000b568     AccessInfo.obj
 0002:00001590       $SG47343                   000000014000b590     AccessInfo.obj
 0002:000015d0       $SG47346                   000000014000b5d0     AccessInfo.obj
 0002:000015f0       $SG47348                   000000014000b5f0     AccessInfo.obj
 0002:00001610       $SG47349                   000000014000b610     AccessInfo.obj
 0002:00001628       $SG47350                   000000014000b628     AccessInfo.obj
 0002:00001644       $SG47352                   000000014000b644     AccessInfo.obj
 0002:00001650       $SG47353                   000000014000b650     AccessInfo.obj
 0002:00001660       $SG47354                   000000014000b660     AccessInfo.obj
 0002:00001680       $SG47355                   000000014000b680     AccessInfo.obj
 0002:00001688       $SG47356                   000000014000b688     AccessInfo.obj
 0002:00001694       $SG47357                   000000014000b694     AccessInfo.obj
 0002:000016a0       $SG47358                   000000014000b6a0     AccessInfo.obj
 0002:000016b0       $SG47359                   000000014000b6b0     AccessInfo.obj
 0002:000016c0       $SG47360                   000000014000b6c0     AccessInfo.obj
 0002:000016c8       $SG47361                   000000014000b6c8     AccessInfo.obj
 0002:000016d8       $SG47362                   000000014000b6d8     AccessInfo.obj
 0002:000016ec       $SG47363                   000000014000b6ec     AccessInfo.obj
 0002:000016f8       $SG47364                   000000014000b6f8     AccessInfo.obj
 0002:00001708       $SG47365                   000000014000b708     AccessInfo.obj
 0002:00001718       $SG47366                   000000014000b718     AccessInfo.obj
 0002:00001720       $SG47367                   000000014000b720     AccessInfo.obj
 0002:00001730       $SG47368                   000000014000b730     AccessInfo.obj
 0002:00001740       $SG47369                   000000014000b740     AccessInfo.obj
 0002:00001748       $SG47370                   000000014000b748     AccessInfo.obj
 0002:00001770       $SG47371                   000000014000b770     AccessInfo.obj
 0002:00001798       $SG47372                   000000014000b798     AccessInfo.obj
 0002:000017b8       $SG47373                   000000014000b7b8     AccessInfo.obj
 0002:000017d8       $SG47374                   000000014000b7d8     AccessInfo.obj
 0002:00001800       $SG47375                   000000014000b800     AccessInfo.obj
 0002:00001820       $SG47376                   000000014000b820     AccessInfo.obj
 0002:00001840       $SG47377                   000000014000b840     AccessInfo.obj
 0002:00001860       $SG47378                   000000014000b860     AccessInfo.obj
 0002:00001880       $SG47379                   000000014000b880     AccessInfo.obj
 0002:000018a0       $SG47380                   000000014000b8a0     AccessInfo.obj
 0002:000018c8       $SG47383                   000000014000b8c8     AccessInfo.obj
 0002:000018e8       $SG47384                   000000014000b8e8     AccessInfo.obj
 0002:00001918       $SG47385                   000000014000b918     AccessInfo.obj
 0002:00001938       $SG47387                   000000014000b938     AccessInfo.obj
 0002:00001970       $SG47389                   000000014000b970     AccessInfo.obj
 0002:000019b0       $SG47392                   000000014000b9b0     AccessInfo.obj
 0002:000019d0       $SG47394                   000000014000b9d0     AccessInfo.obj
 0002:000019f0       $SG47395                   000000014000b9f0     AccessInfo.obj
 0002:00001a08       $SG47396                   000000014000ba08     AccessInfo.obj
 0002:00001a24       $SG47398                   000000014000ba24     AccessInfo.obj
 0002:00001a30       $SG47399                   000000014000ba30     AccessInfo.obj
 0002:00001a40       $SG47400                   000000014000ba40     AccessInfo.obj
 0002:00001a60       $SG47401                   000000014000ba60     AccessInfo.obj
 0002:00001a68       $SG47402                   000000014000ba68     AccessInfo.obj
 0002:00001a74       $SG47403                   000000014000ba74     AccessInfo.obj
 0002:00001a80       $SG47404                   000000014000ba80     AccessInfo.obj
 0002:00001a90       $SG47405                   000000014000ba90     AccessInfo.obj
 0002:00001aa0       $SG47406                   000000014000baa0     AccessInfo.obj
 0002:00001aa8       $SG47407                   000000014000baa8     AccessInfo.obj
 0002:00001ab8       $SG47408                   000000014000bab8     AccessInfo.obj
 0002:00001acc       $SG47409                   000000014000bacc     AccessInfo.obj
 0002:00001ad8       $SG47410                   000000014000bad8     AccessInfo.obj
 0002:00001ae8       $SG47411                   000000014000bae8     AccessInfo.obj
 0002:00001af8       $SG47412                   000000014000baf8     AccessInfo.obj
 0002:00001b00       $SG47413                   000000014000bb00     AccessInfo.obj
 0002:00001b10       $SG47414                   000000014000bb10     AccessInfo.obj
 0002:00001b20       $SG47415                   000000014000bb20     AccessInfo.obj
 0002:00001b28       $SG47416                   000000014000bb28     AccessInfo.obj
 0002:00001b50       $SG47417                   000000014000bb50     AccessInfo.obj
 0002:00001b78       $SG47418                   000000014000bb78     AccessInfo.obj
 0002:00001b98       $SG47419                   000000014000bb98     AccessInfo.obj
 0002:00001bb8       $SG47420                   000000014000bbb8     AccessInfo.obj
 0002:00001be0       $SG47421                   000000014000bbe0     AccessInfo.obj
 0002:00001c00       $SG47422                   000000014000bc00     AccessInfo.obj
 0002:00001c20       $SG47423                   000000014000bc20     AccessInfo.obj
 0002:00001c40       $SG47424                   000000014000bc40     AccessInfo.obj
 0002:00001c60       $SG47425                   000000014000bc60     AccessInfo.obj
 0002:00001c80       $SG47426                   000000014000bc80     AccessInfo.obj
 0002:00001ca8       $SG47429                   000000014000bca8     AccessInfo.obj
 0002:00001cc8       $SG47430                   000000014000bcc8     AccessInfo.obj
 0002:00001d00       $SG54777                   000000014000bd00     jaccesswalker.obj
 0002:00001d02       $SG54825                   000000014000bd02     jaccesswalker.obj
 0002:00001d03       $SG54899                   000000014000bd03     jaccesswalker.obj
 0002:00001d04       $SG55002                   000000014000bd04     jaccesswalker.obj
 0002:00001d08       $SG54778                   000000014000bd08     jaccesswalker.obj
 0002:00001d20       $SG54779                   000000014000bd20     jaccesswalker.obj
 0002:00001d40       $SG54865                   000000014000bd40     jaccesswalker.obj
 0002:00001d4c       $SG54900                   000000014000bd4c     jaccesswalker.obj
 0002:00001d58       $SG54928                   000000014000bd58     jaccesswalker.obj
 0002:00001d60       $SG54929                   000000014000bd60     jaccesswalker.obj
 0002:00001d78       $SG54952                   000000014000bd78     jaccesswalker.obj
 0002:00001d88       $SG54959                   000000014000bd88     jaccesswalker.obj
 0002:00001d98       $SG54963                   000000014000bd98     jaccesswalker.obj
 0002:00001da8       $SG54965                   000000014000bda8     jaccesswalker.obj
 0002:00001db8       $SG54968                   000000014000bdb8     jaccesswalker.obj
 0002:00001dc8       $SG54970                   000000014000bdc8     jaccesswalker.obj
 0002:00001dd8       $SG54972                   000000014000bdd8     jaccesswalker.obj
 0002:00001de8       $SG54977                   000000014000bde8     jaccesswalker.obj
 0002:00001df8       $SG54979                   000000014000bdf8     jaccesswalker.obj
 0002:00001e08       $SG54982                   000000014000be08     jaccesswalker.obj
 0002:00001e18       $SG55003                   000000014000be18     jaccesswalker.obj
 0002:00001e28       $SG55050                   000000014000be28     jaccesswalker.obj
 0002:00001e2c       $SG55051                   000000014000be2c     jaccesswalker.obj
 0002:00001e30       $SG55052                   000000014000be30     jaccesswalker.obj
 0002:00001e40       $SG55053                   000000014000be40     jaccesswalker.obj
 0002:00001e88       $SG55083                   000000014000be88     jaccesswalker.obj
 0002:00001ea8       $SG55085                   000000014000bea8     jaccesswalker.obj
 0002:00001ec8       GS_ExceptionPointers       000000014000bec8     MSVCRT:gs_report.obj
 0002:00002780       $unwind$initializeAccessBridge 000000014000c780     AccessBridgeCalls.obj
 0002:00002788       $unwind$shutdownAccessBridge 000000014000c788     AccessBridgeCalls.obj
 0002:00002790       $unwind$IsJavaWindow       000000014000c790     AccessBridgeCalls.obj
 0002:00002798       $unwind$GetAccessibleContextFromHWND 000000014000c798     AccessBridgeCalls.obj
 0002:000027a0       $unwind$getHWNDFromAccessibleContext 000000014000c7a0     AccessBridgeCalls.obj
 0002:000027a8       $unwind$SetJavaShutdown    000000014000c7a8     AccessBridgeCalls.obj
 0002:000027b0       $unwind$SetFocusGained     000000014000c7b0     AccessBridgeCalls.obj
 0002:000027b8       $unwind$SetFocusLost       000000014000c7b8     AccessBridgeCalls.obj
 0002:000027c0       $unwind$SetCaretUpdate     000000014000c7c0     AccessBridgeCalls.obj
 0002:000027c8       $unwind$SetMouseClicked    000000014000c7c8     AccessBridgeCalls.obj
 0002:000027d0       $unwind$SetMouseEntered    000000014000c7d0     AccessBridgeCalls.obj
 0002:000027d8       $unwind$SetMouseExited     000000014000c7d8     AccessBridgeCalls.obj
 0002:000027e0       $unwind$SetMousePressed    000000014000c7e0     AccessBridgeCalls.obj
 0002:000027e8       $unwind$SetMouseReleased   000000014000c7e8     AccessBridgeCalls.obj
 0002:000027f0       $unwind$SetMenuCanceled    000000014000c7f0     AccessBridgeCalls.obj
 0002:000027f8       $unwind$SetMenuDeselected  000000014000c7f8     AccessBridgeCalls.obj
 0002:00002800       $unwind$SetMenuSelected    000000014000c800     AccessBridgeCalls.obj
 0002:00002808       $unwind$SetPopupMenuCanceled 000000014000c808     AccessBridgeCalls.obj
 0002:00002810       $unwind$SetPopupMenuWillBecomeInvisible 000000014000c810     AccessBridgeCalls.obj
 0002:00002818       $unwind$SetPopupMenuWillBecomeVisible 000000014000c818     AccessBridgeCalls.obj
 0002:00002820       $unwind$SetPropertyNameChange 000000014000c820     AccessBridgeCalls.obj
 0002:00002828       $unwind$SetPropertyDescriptionChange 000000014000c828     AccessBridgeCalls.obj
 0002:00002830       $unwind$SetPropertyStateChange 000000014000c830     AccessBridgeCalls.obj
 0002:00002838       $unwind$SetPropertyValueChange 000000014000c838     AccessBridgeCalls.obj
 0002:00002840       $unwind$SetPropertySelectionChange 000000014000c840     AccessBridgeCalls.obj
 0002:00002848       $unwind$SetPropertyTextChange 000000014000c848     AccessBridgeCalls.obj
 0002:00002850       $unwind$SetPropertyCaretChange 000000014000c850     AccessBridgeCalls.obj
 0002:00002858       $unwind$SetPropertyVisibleDataChange 000000014000c858     AccessBridgeCalls.obj
 0002:00002860       $unwind$SetPropertyChildChange 000000014000c860     AccessBridgeCalls.obj
 0002:00002868       $unwind$SetPropertyActiveDescendentChange 000000014000c868     AccessBridgeCalls.obj
 0002:00002870       $unwind$SetPropertyTableModelChange 000000014000c870     AccessBridgeCalls.obj
 0002:00002878       $unwind$ReleaseJavaObject  000000014000c878     AccessBridgeCalls.obj
 0002:00002880       $unwind$GetVersionInfo     000000014000c880     AccessBridgeCalls.obj
 0002:00002888       $unwind$GetAccessibleContextAt 000000014000c888     AccessBridgeCalls.obj
 0002:00002890       $unwind$GetAccessibleContextWithFocus 000000014000c890     AccessBridgeCalls.obj
 0002:00002898       $unwind$GetAccessibleContextInfo 000000014000c898     AccessBridgeCalls.obj
 0002:000028a0       $unwind$GetAccessibleChildFromContext 000000014000c8a0     AccessBridgeCalls.obj
 0002:000028a8       $unwind$GetAccessibleParentFromContext 000000014000c8a8     AccessBridgeCalls.obj
 0002:000028b0       $unwind$GetAccessibleTextInfo 000000014000c8b0     AccessBridgeCalls.obj
 0002:000028b8       $unwind$GetAccessibleTextItems 000000014000c8b8     AccessBridgeCalls.obj
 0002:000028c0       $unwind$GetAccessibleTextSelectionInfo 000000014000c8c0     AccessBridgeCalls.obj
 0002:000028c8       $unwind$GetAccessibleTextAttributes 000000014000c8c8     AccessBridgeCalls.obj
 0002:000028d0       $unwind$GetAccessibleTextRect 000000014000c8d0     AccessBridgeCalls.obj
 0002:000028d8       $unwind$GetAccessibleTextLineBounds 000000014000c8d8     AccessBridgeCalls.obj
 0002:000028e0       $unwind$GetAccessibleTextRange 000000014000c8e0     AccessBridgeCalls.obj
 0002:000028e8       $unwind$getAccessibleTableInfo 000000014000c8e8     AccessBridgeCalls.obj
 0002:000028f0       $unwind$getAccessibleTableCellInfo 000000014000c8f0     AccessBridgeCalls.obj
 0002:000028f8       $unwind$getAccessibleTableRowHeader 000000014000c8f8     AccessBridgeCalls.obj
 0002:00002900       $unwind$getAccessibleTableColumnHeader 000000014000c900     AccessBridgeCalls.obj
 0002:00002908       $unwind$getAccessibleTableRowDescription 000000014000c908     AccessBridgeCalls.obj
 0002:00002910       $unwind$getAccessibleTableColumnDescription 000000014000c910     AccessBridgeCalls.obj
 0002:00002918       $unwind$getAccessibleTableRowSelectionCount 000000014000c918     AccessBridgeCalls.obj
 0002:00002920       $unwind$isAccessibleTableRowSelected 000000014000c920     AccessBridgeCalls.obj
 0002:00002928       $unwind$getAccessibleTableRowSelections 000000014000c928     AccessBridgeCalls.obj
 0002:00002930       $unwind$getAccessibleTableColumnSelectionCount 000000014000c930     AccessBridgeCalls.obj
 0002:00002938       $unwind$isAccessibleTableColumnSelected 000000014000c938     AccessBridgeCalls.obj
 0002:00002940       $unwind$getAccessibleTableColumnSelections 000000014000c940     AccessBridgeCalls.obj
 0002:00002948       $unwind$getAccessibleTableRow 000000014000c948     AccessBridgeCalls.obj
 0002:00002950       $unwind$getAccessibleTableColumn 000000014000c950     AccessBridgeCalls.obj
 0002:00002958       $unwind$getAccessibleTableIndex 000000014000c958     AccessBridgeCalls.obj
 0002:00002960       $unwind$getAccessibleRelationSet 000000014000c960     AccessBridgeCalls.obj
 0002:00002968       $unwind$getAccessibleHypertext 000000014000c968     AccessBridgeCalls.obj
 0002:00002970       $unwind$activateAccessibleHyperlink 000000014000c970     AccessBridgeCalls.obj
 0002:00002978       $unwind$getAccessibleHyperlinkCount 000000014000c978     AccessBridgeCalls.obj
 0002:00002980       $unwind$getAccessibleHypertextExt 000000014000c980     AccessBridgeCalls.obj
 0002:00002988       $unwind$getAccessibleHypertextLinkIndex 000000014000c988     AccessBridgeCalls.obj
 0002:00002990       $unwind$getAccessibleHyperlink 000000014000c990     AccessBridgeCalls.obj
 0002:00002998       $unwind$getAccessibleKeyBindings 000000014000c998     AccessBridgeCalls.obj
 0002:000029a0       $unwind$getAccessibleIcons 000000014000c9a0     AccessBridgeCalls.obj
 0002:000029a8       $unwind$getAccessibleActions 000000014000c9a8     AccessBridgeCalls.obj
 0002:000029b0       $unwind$doAccessibleActions 000000014000c9b0     AccessBridgeCalls.obj
 0002:000029b8       $unwind$IsSameObject       000000014000c9b8     AccessBridgeCalls.obj
 0002:000029c0       $unwind$setTextContents    000000014000c9c0     AccessBridgeCalls.obj
 0002:000029c8       $unwind$getParentWithRole  000000014000c9c8     AccessBridgeCalls.obj
 0002:000029d0       $unwind$getParentWithRoleElseRoot 000000014000c9d0     AccessBridgeCalls.obj
 0002:000029d8       $unwind$getTopLevelObject  000000014000c9d8     AccessBridgeCalls.obj
 0002:000029e0       $unwind$getObjectDepth     000000014000c9e0     AccessBridgeCalls.obj
 0002:000029e8       $unwind$getActiveDescendent 000000014000c9e8     AccessBridgeCalls.obj
 0002:000029f0       $unwind$GetCurrentAccessibleValueFromContext 000000014000c9f0     AccessBridgeCalls.obj
 0002:000029f8       $unwind$GetMaximumAccessibleValueFromContext 000000014000c9f8     AccessBridgeCalls.obj
 0002:00002a00       $unwind$GetMinimumAccessibleValueFromContext 000000014000ca00     AccessBridgeCalls.obj
 0002:00002a08       $unwind$GetAccessibleSelectionFromContext 000000014000ca08     AccessBridgeCalls.obj
 0002:00002a10       $unwind$GetAccessibleSelectionCountFromContext 000000014000ca10     AccessBridgeCalls.obj
 0002:00002a18       $unwind$IsAccessibleChildSelectedFromContext 000000014000ca18     AccessBridgeCalls.obj
 0002:00002a20       $unwind$RemoveAccessibleSelectionFromContext 000000014000ca20     AccessBridgeCalls.obj
 0002:00002a28       $unwind$SelectAllAccessibleSelectionFromContext 000000014000ca28     AccessBridgeCalls.obj
 0002:00002a30       $unwind$getVirtualAccessibleName 000000014000ca30     AccessBridgeCalls.obj
 0002:00002a38       $unwind$requestFocus       000000014000ca38     AccessBridgeCalls.obj
 0002:00002a40       $unwind$selectTextRange    000000014000ca40     AccessBridgeCalls.obj
 0002:00002a48       $unwind$getTextAttributesInRange 000000014000ca48     AccessBridgeCalls.obj
 0002:00002a50       $unwind$getVisibleChildrenCount 000000014000ca50     AccessBridgeCalls.obj
 0002:00002a58       $unwind$getVisibleChildren 000000014000ca58     AccessBridgeCalls.obj
 0002:00002a60       $unwind$setCaretPosition   000000014000ca60     AccessBridgeCalls.obj
 0002:00002a68       $unwind$getCaretLocation   000000014000ca68     AccessBridgeCalls.obj
 0002:00002a70       $unwind$getEventsWaiting   000000014000ca70     AccessBridgeCalls.obj
 0002:00002a78       $unwind$addAccessibleSelectionFromContext 000000014000ca78     AccessBridgeCalls.obj
 0002:00002a80       $unwind$clearAccessibleSelectionFromContext 000000014000ca80     AccessBridgeCalls.obj
 0002:00002a88       $unwind$printError         000000014000ca88     AccessBridgeDebug.obj
 0002:00002a90       $unwind$PrintDebugString   000000014000ca90     AccessBridgeDebug.obj
 0002:00002a98       $unwind$wPrintJavaDebugString 000000014000ca98     AccessBridgeDebug.obj
 0002:00002aa0       $unwind$wPrintDebugString  000000014000caa0     AccessBridgeDebug.obj
 0002:00002aa8       $unwind$initializeFileLogger 000000014000caa8     AccessBridgeDebug.obj
 0002:00002ab0       $unwind$finalizeFileLogger 000000014000cab0     AccessBridgeDebug.obj
 0002:00002ab8       $unwind$getTimeStamp       000000014000cab8     AccessBridgeDebug.obj
 0002:00002ac0       $unwind$PrintJavaDebugString2 000000014000cac0     AccessBridgeDebug.obj
 0002:00002ac8       $unwind$_vfprintf_l        000000014000cac8     AccessBridgeDebug.obj
 0002:00002ac8       $unwind$_vfwprintf_l       000000014000cac8     AccessBridgeDebug.obj
 0002:00002ac8       $unwind$fprintf            000000014000cac8     AccessBridgeDebug.obj
 0002:00002ac8       $unwind$printf             000000014000cac8     AccessBridgeDebug.obj
 0002:00002ac8       $unwind$snprintf           000000014000cac8     AccessInfo.obj
 0002:00002ad0       $unwind$vfprintf           000000014000cad0     AccessBridgeDebug.obj
 0002:00002ad0       $unwind$vfwprintf          000000014000cad0     AccessBridgeDebug.obj
 0002:00002ad8       $unwind$?initBroadcastMessageIDs@@YAHXZ 000000014000cad8     AccessBridgeMessages.obj
 0002:00002ae0       $unwind$vsnprintf          000000014000cae0     AccessInfo.obj
 0002:00002ae8       $unwind$?getTimeAndDate@@YAPEADXZ 000000014000cae8     AccessInfo.obj
 0002:00002af4       $unwind$?displayAndLog@@YAXPEAUHWND__@@HPEAU_iobuf@@PEADZZ 000000014000caf4     AccessInfo.obj
 0002:00002b04       $unwind$?logString@@YAXPEAU_iobuf@@PEBDZZ 000000014000cb04     AccessInfo.obj
 0002:00002b14       $unwind$?getAccessibleInfo@@YAPEADJ_JPEADH@Z 000000014000cb14     AccessInfo.obj
 0002:00002b1c       $unwind$?getAccessibleInfo@@YAPEADJ_JHHPEADH@Z 000000014000cb1c     AccessInfo.obj
 0002:00002b30       $unwind$localtime          000000014000cb30     AccessInfo.obj
 0002:00002b38       $unwind$time               000000014000cb38     AccessInfo.obj
 0002:00002b40       $unwind$?appendToBuffer@@YAHPEAD_KPEBDZZ 000000014000cb40     AccessInfo.obj
 0002:00002b50       $unwind$WinMain            000000014000cb50     jaccesswalker.obj
 0002:00002b58       $unwind$??1AccessibleNode@@QEAA@XZ 000000014000cb58     jaccesswalker.obj
 0002:00002b60       $unwind$?setAccessibleName@AccessibleNode@@QEAAXPEAD@Z 000000014000cb60     jaccesswalker.obj
 0002:00002b68       $unwind$?setAccessibleRole@AccessibleNode@@QEAAXPEAD@Z 000000014000cb68     jaccesswalker.obj
 0002:00002b70       $unwind$?displayAPIWindow@AccessibleNode@@QEAAHXZ 000000014000cb70     jaccesswalker.obj
 0002:00002b80       $unwind$??0Jaccesswalker@@QEAA@H@Z 000000014000cb80     jaccesswalker.obj
 0002:00002b88       $unwind$?buildAccessibilityTree@Jaccesswalker@@QEAAXXZ 000000014000cb88     jaccesswalker.obj
 0002:00002b90       $unwind$?addComponentNodes@Jaccesswalker@@QEAAXJ_JPEAVAccessibleNode@@PEAUHWND__@@PEAU_TREEITEM@@2@Z 000000014000cb90     jaccesswalker.obj
 0002:00002ba8       $cppxdata$?addComponentNodes@Jaccesswalker@@QEAAXJ_JPEAVAccessibleNode@@PEAUHWND__@@PEAU_TREEITEM@@2@Z 000000014000cba8     jaccesswalker.obj
 0002:00002bb1       $stateUnwindMap$?addComponentNodes@Jaccesswalker@@QEAAXJ_JPEAVAccessibleNode@@PEAUHWND__@@PEAU_TREEITEM@@2@Z 000000014000cbb1     jaccesswalker.obj
 0002:00002bb7       $ip2state$?addComponentNodes@Jaccesswalker@@QEAAXJ_JPEAVAccessibleNode@@PEAUHWND__@@PEAU_TREEITEM@@2@Z 000000014000cbb7     jaccesswalker.obj
 0002:00002bc0       $unwind$?dtor$0@?0??addComponentNodes@Jaccesswalker@@QEAAXJ_JPEAVAccessibleNode@@PEAUHWND__@@PEAU_TREEITEM@@2@Z@4HA 000000014000cbc0     jaccesswalker.obj
 0002:00002bc8       $unwind$?WinProc@@YA_JPEAUHWND__@@I_K_J@Z 000000014000cbc8     jaccesswalker.obj
 0002:00002bd0       $unwind$?EnumWndProc@@YAHPEAUHWND__@@_J@Z 000000014000cbd0     jaccesswalker.obj
 0002:00002be4       $unwind$?EnumChildProc@@YAHPEAUHWND__@@_J@Z 000000014000cbe4     jaccesswalker.obj
 0002:00002bec       $unwind$?CreateATreeView@@YAPEAUHWND__@@PEAU1@@Z 000000014000cbec     jaccesswalker.obj
 0002:00002bfc       $unwind$?AccessInfoWindowProc@@YA_JPEAUHWND__@@IIJ@Z 000000014000cbfc     jaccesswalker.obj
 0002:00002c0c       $unwind$?IsInaccessibleJavaWindow@@YAHQEAUHWND__@@@Z 000000014000cc0c     jaccesswalker.obj
 0002:00002c20       $unwind$__report_securityfailure 000000014000cc20     MSVCRT:gs_report.obj
 0002:00002c28       $unwind$__scrt_initialize_default_local_stdio_options 000000014000cc28     MSVCRT:default_local_stdio_options.obj
 0002:00002c28       $unwind$?post_pgo_initialization@@YAHXZ 000000014000cc28     MSVCRT:exe_winmain.obj
 0002:00002c28       $unwind$?pre_cpp_initialization@@YAXXZ 000000014000cc28     MSVCRT:exe_winmain.obj
 0002:00002c28       $unwind$WinMainCRTStartup  000000014000cc28     MSVCRT:exe_winmain.obj
 0002:00002c28       $unwind$__report_rangecheckfailure 000000014000cc28     MSVCRT:gs_report.obj
 0002:00002c28       $unwind$__GSHandlerCheck   000000014000cc28     MSVCRT:gshandler.obj
 0002:00002c28       $unwind$__scrt_acquire_startup_lock 000000014000cc28     MSVCRT:utility.obj
 0002:00002c28       $unwind$atexit             000000014000cc28     MSVCRT:utility.obj
 0002:00002c28       $unwind$__scrt_is_managed_app 000000014000cc28     MSVCRT:utility_desktop.obj
 0002:00002c30       $unwind$__report_gsfailure 000000014000cc30     MSVCRT:gs_report.obj
 0002:00002c38       $unwind$capture_current_context 000000014000cc38     MSVCRT:gs_report.obj
 0002:00002c44       $unwind$capture_previous_context 000000014000cc44     MSVCRT:gs_report.obj
 0002:00002c50       $unwind$?pre_c_initialization@@YAHXZ 000000014000cc50     MSVCRT:exe_winmain.obj
 0002:00002c50       $unwind$__raise_securityfailure 000000014000cc50     MSVCRT:gs_report.obj
 0002:00002c50       $unwind$??2@YAPEAX_K@Z     000000014000cc50     MSVCRT:new_scalar.obj
 0002:00002c50       $unwind$??_Gtype_info@@UEAAPEAXI@Z 000000014000cc50     MSVCRT:std_type_info_static.obj
 0002:00002c50       $unwind$??0bad_alloc@std@@QEAA@AEBV01@@Z 000000014000cc50     MSVCRT:throw_bad_alloc.obj
 0002:00002c50       $unwind$??0bad_array_new_length@std@@QEAA@AEBV01@@Z 000000014000cc50     MSVCRT:throw_bad_alloc.obj
 0002:00002c50       $unwind$??0exception@std@@QEAA@AEBV01@@Z 000000014000cc50     MSVCRT:throw_bad_alloc.obj
 0002:00002c50       $unwind$__scrt_initialize_crt 000000014000cc50     MSVCRT:utility.obj
 0002:00002c50       $unwind$__scrt_initialize_onexit_tables 000000014000cc50     MSVCRT:utility.obj
 0002:00002c50       $unwind$__scrt_release_startup_lock 000000014000cc50     MSVCRT:utility.obj
 0002:00002c50       $unwind$__scrt_uninitialize_crt 000000014000cc50     MSVCRT:utility.obj
 0002:00002c50       $unwind$_onexit            000000014000cc50     MSVCRT:utility.obj
 0002:00002c58       $unwind$__GSHandlerCheckCommon 000000014000cc58     MSVCRT:gshandler.obj
 0002:00002c60       $xdatasym                  000000014000cc60     MSVCRT:chkstk.obj
 0002:00002c68       $xdatasym                  000000014000cc68     MSVCRT:amdsecgs.obj
 0002:00002c6c       $unwind$__GSHandlerCheck_EH4 000000014000cc6c     MSVCRT:gshandlereh4.obj
 0002:00002c84       $unwind$?__scrt_common_main_seh@@YAHXZ 000000014000cc84     MSVCRT:exe_winmain.obj
 0002:00002cb8       $unwind$?filt$0@?0??__scrt_common_main_seh@@YAHXZ@4HA 000000014000ccb8     MSVCRT:exe_winmain.obj
 0002:00002cc0       $unwind$_RTC_Initialize    000000014000ccc0     MSVCRT:initsect.obj
 0002:00002cc0       $unwind$_RTC_Terminate     000000014000ccc0     MSVCRT:initsect.obj
 0002:00002cc0       $unwind$??_Gbad_alloc@std@@UEAAPEAXI@Z 000000014000ccc0     MSVCRT:throw_bad_alloc.obj
 0002:00002cc0       $unwind$??_Gbad_array_new_length@std@@UEAAPEAXI@Z 000000014000ccc0     MSVCRT:throw_bad_alloc.obj
 0002:00002cc0       $unwind$??_Gexception@std@@UEAAPEAXI@Z 000000014000ccc0     MSVCRT:throw_bad_alloc.obj
 0002:00002cc0       $unwind$__scrt_unhandled_exception_filter 000000014000ccc0     MSVCRT:utility_desktop.obj
 0002:00002ccc       $unwind$?__scrt_throw_std_bad_alloc@@YAXXZ 000000014000cccc     MSVCRT:throw_bad_alloc.obj
 0002:00002ccc       $unwind$?__scrt_throw_std_bad_array_new_length@@YAXXZ 000000014000cccc     MSVCRT:throw_bad_alloc.obj
 0002:00002cd4       $unwind$__scrt_is_nonwritable_in_current_image 000000014000ccd4     MSVCRT:utility.obj
 0002:00002cf4       $unwind$__scrt_is_nonwritable_in_current_image$filt$0 000000014000ccf4     MSVCRT:utility.obj
 0002:00002cfc       $unwind$__security_init_cookie 000000014000ccfc     MSVCRT:gs_support.obj
 0002:00002d08       $unwind$__scrt_get_show_window_mode 000000014000cd08     MSVCRT:utility_desktop.obj
 0002:00002d10       $unwind$__scrt_fastfail    000000014000cd10     MSVCRT:utility_desktop.obj
 0002:00002d20       $unwind$__isa_available_init 000000014000cd20     MSVCRT:cpu_disp.obj
 0002:00002d30       $xdatasym                  000000014000cd30     MSVCRT:guard_dispatch.obj
 0002:00002d38       $xdatasym                  000000014000cd38     MSVCRT:guard_xfg_dispatch.obj
 0002:00003310       .idata$6                   000000014000d310     comctl32:COMCTL32.dll
 0002:00003330       .idata$6                   000000014000d330     gdi32:GDI32.dll
 0002:00003504       .idata$6                   000000014000d504     user32:USER32.dll
 0002:000036de       .idata$6                   000000014000d6de     kernel32:KERNEL32.dll
 0002:000037aa       .idata$6                   000000014000d7aa     vcruntime:VCRUNTIME140.dll
 0002:000037bc       .idata$6                   000000014000d7bc     vcruntime:VCRUNTIME140_1.dll
 0002:00003a6e       .idata$6                   000000014000da6e     ucrt:api-ms-win-crt-string-l1-1-0.dll
 0002:00003a90       .idata$6                   000000014000da90     ucrt:api-ms-win-crt-stdio-l1-1-0.dll
 0002:00003ab0       .idata$6                   000000014000dab0     ucrt:api-ms-win-crt-environment-l1-1-0.dll
 0002:00003ad6       .idata$6                   000000014000dad6     ucrt:api-ms-win-crt-time-l1-1-0.dll
 0002:00003af6       .idata$6                   000000014000daf6     ucrt:api-ms-win-crt-heap-l1-1-0.dll
 0002:00003b16       .idata$6                   000000014000db16     ucrt:api-ms-win-crt-runtime-l1-1-0.dll
 0002:00003b38       .idata$6                   000000014000db38     ucrt:api-ms-win-crt-math-l1-1-0.dll
 0002:00003b58       .idata$6                   000000014000db58     ucrt:api-ms-win-crt-locale-l1-1-0.dll
 0003:00000000       $SG37390                   000000014000e000     AccessBridgeCalls.obj
 0003:00000018       $SG37394                   000000014000e018     AccessBridgeCalls.obj
 0003:00000028       $SG37396                   000000014000e028     AccessBridgeCalls.obj
 0003:00000040       $SG37398                   000000014000e040     AccessBridgeCalls.obj
 0003:00000058       $SG37400                   000000014000e058     AccessBridgeCalls.obj
 0003:00000068       $SG37402                   000000014000e068     AccessBridgeCalls.obj
 0003:00000080       $SG37404                   000000014000e080     AccessBridgeCalls.obj
 0003:00000098       $SG37406                   000000014000e098     AccessBridgeCalls.obj
 0003:000000b0       $SG37408                   000000014000e0b0     AccessBridgeCalls.obj
 0003:000000c8       $SG37410                   000000014000e0c8     AccessBridgeCalls.obj
 0003:000000e0       $SG37412                   000000014000e0e0     AccessBridgeCalls.obj
 0003:000000f8       $SG37414                   000000014000e0f8     AccessBridgeCalls.obj
 0003:00000110       $SG37416                   000000014000e110     AccessBridgeCalls.obj
 0003:00000128       $SG37418                   000000014000e128     AccessBridgeCalls.obj
 0003:00000140       $SG37420                   000000014000e140     AccessBridgeCalls.obj
 0003:00000158       $SG37422                   000000014000e158     AccessBridgeCalls.obj
 0003:00000180       $SG37424                   000000014000e180     AccessBridgeCalls.obj
 0003:000001a0       $SG37426                   000000014000e1a0     AccessBridgeCalls.obj
 0003:000001b8       $SG37428                   000000014000e1b8     AccessBridgeCalls.obj
 0003:000001d8       $SG37430                   000000014000e1d8     AccessBridgeCalls.obj
 0003:000001f8       $SG37432                   000000014000e1f8     AccessBridgeCalls.obj
 0003:00000218       $SG37434                   000000014000e218     AccessBridgeCalls.obj
 0003:00000238       $SG37436                   000000014000e238     AccessBridgeCalls.obj
 0003:00000250       $SG37438                   000000014000e250     AccessBridgeCalls.obj
 0003:00000270       $SG37440                   000000014000e270     AccessBridgeCalls.obj
 0003:00000290       $SG37442                   000000014000e290     AccessBridgeCalls.obj
 0003:000002b0       $SG37444                   000000014000e2b0     AccessBridgeCalls.obj
 0003:000002d8       $SG37446                   000000014000e2d8     AccessBridgeCalls.obj
 0003:000002f8       $SG37448                   000000014000e2f8     AccessBridgeCalls.obj
 0003:00000310       $SG37450                   000000014000e310     AccessBridgeCalls.obj
 0003:00000320       $SG37452                   000000014000e320     AccessBridgeCalls.obj
 0003:00000330       $SG37454                   000000014000e330     AccessBridgeCalls.obj
 0003:00000340       $SG37456                   000000014000e340     AccessBridgeCalls.obj
 0003:00000360       $SG37458                   000000014000e360     AccessBridgeCalls.obj
 0003:00000380       $SG37460                   000000014000e380     AccessBridgeCalls.obj
 0003:00000398       $SG37462                   000000014000e398     AccessBridgeCalls.obj
 0003:000003b8       $SG37464                   000000014000e3b8     AccessBridgeCalls.obj
 0003:000003d8       $SG37466                   000000014000e3d8     AccessBridgeCalls.obj
 0003:000003f8       $SG37468                   000000014000e3f8     AccessBridgeCalls.obj
 0003:00000418       $SG37470                   000000014000e418     AccessBridgeCalls.obj
 0003:00000430       $SG37472                   000000014000e430     AccessBridgeCalls.obj
 0003:00000450       $SG37474                   000000014000e450     AccessBridgeCalls.obj
 0003:00000470       $SG37476                   000000014000e470     AccessBridgeCalls.obj
 0003:00000490       $SG37478                   000000014000e490     AccessBridgeCalls.obj
 0003:000004b8       $SG37480                   000000014000e4b8     AccessBridgeCalls.obj
 0003:000004e0       $SG37482                   000000014000e4e0     AccessBridgeCalls.obj
 0003:00000508       $SG37484                   000000014000e508     AccessBridgeCalls.obj
 0003:00000528       $SG37486                   000000014000e528     AccessBridgeCalls.obj
 0003:00000548       $SG37488                   000000014000e548     AccessBridgeCalls.obj
 0003:00000570       $SG37490                   000000014000e570     AccessBridgeCalls.obj
 0003:00000590       $SG37492                   000000014000e590     AccessBridgeCalls.obj
 0003:000005b8       $SG37494                   000000014000e5b8     AccessBridgeCalls.obj
 0003:000005d0       $SG37496                   000000014000e5d0     AccessBridgeCalls.obj
 0003:000005f0       $SG37498                   000000014000e5f0     AccessBridgeCalls.obj
 0003:00000608       $SG37500                   000000014000e608     AccessBridgeCalls.obj
 0003:00000628       $SG37502                   000000014000e628     AccessBridgeCalls.obj
 0003:00000640       $SG37504                   000000014000e640     AccessBridgeCalls.obj
 0003:00000660       $SG37506                   000000014000e660     AccessBridgeCalls.obj
 0003:00000680       $SG37508                   000000014000e680     AccessBridgeCalls.obj
 0003:000006a0       $SG37510                   000000014000e6a0     AccessBridgeCalls.obj
 0003:000006c0       $SG37512                   000000014000e6c0     AccessBridgeCalls.obj
 0003:000006d8       $SG37514                   000000014000e6d8     AccessBridgeCalls.obj
 0003:000006f8       $SG37516                   000000014000e6f8     AccessBridgeCalls.obj
 0003:00000710       $SG37518                   000000014000e710     AccessBridgeCalls.obj
 0003:00000728       $SG37520                   000000014000e728     AccessBridgeCalls.obj
 0003:00000740       $SG37522                   000000014000e740     AccessBridgeCalls.obj
 0003:00000758       $SG37524                   000000014000e758     AccessBridgeCalls.obj
 0003:00000770       $SG37526                   000000014000e770     AccessBridgeCalls.obj
 0003:00000790       $SG37528                   000000014000e790     AccessBridgeCalls.obj
 0003:000007b0       $SG37530                   000000014000e7b0     AccessBridgeCalls.obj
 0003:000007c8       $SG37532                   000000014000e7c8     AccessBridgeCalls.obj
 0003:000007e8       $SG37534                   000000014000e7e8     AccessBridgeCalls.obj
 0003:00000800       $SG37536                   000000014000e800     AccessBridgeCalls.obj
 0003:00000828       $SG37538                   000000014000e828     AccessBridgeCalls.obj
 0003:00000850       $SG37540                   000000014000e850     AccessBridgeCalls.obj
 0003:00000878       $SG37542                   000000014000e878     AccessBridgeCalls.obj
 0003:000008a0       $SG37544                   000000014000e8a0     AccessBridgeCalls.obj
 0003:000008c8       $SG37546                   000000014000e8c8     AccessBridgeCalls.obj
 0003:000008f0       $SG37548                   000000014000e8f0     AccessBridgeCalls.obj
 0003:00000918       $SG37550                   000000014000e918     AccessBridgeCalls.obj
 0003:00000940       $SG37552                   000000014000e940     AccessBridgeCalls.obj
 0003:00000968       $SG37554                   000000014000e968     AccessBridgeCalls.obj
 0003:00000990       $SG37556                   000000014000e990     AccessBridgeCalls.obj
 0003:000009a0       $SG37558                   000000014000e9a0     AccessBridgeCalls.obj
 0003:000009b8       $SG37560                   000000014000e9b8     AccessBridgeCalls.obj
 0003:000009d0       $SG37562                   000000014000e9d0     AccessBridgeCalls.obj
 0003:000009f0       $SG37564                   000000014000e9f0     AccessBridgeCalls.obj
 0003:00000a00       $SG37566                   000000014000ea00     AccessBridgeCalls.obj
 0003:00000a18       $SG37568                   000000014000ea18     AccessBridgeCalls.obj
 0003:00000a38       $SG37570                   000000014000ea38     AccessBridgeCalls.obj
 0003:00000a48       $SG37572                   000000014000ea48     AccessBridgeCalls.obj
 0003:00000a58       $SG37574                   000000014000ea58     AccessBridgeCalls.obj
 0003:00000a78       $SG37576                   000000014000ea78     AccessBridgeCalls.obj
 0003:00000a90       $SG37578                   000000014000ea90     AccessBridgeCalls.obj
 0003:00000aa8       $SG37580                   000000014000eaa8     AccessBridgeCalls.obj
 0003:00000ac0       $SG37582                   000000014000eac0     AccessBridgeCalls.obj
 0003:00000ad8       $SG37584                   000000014000ead8     AccessBridgeCalls.obj
 0003:00000af0       ?warning@?1??appendToBuffer@@YAHPEAD_KPEBDZZ@4PADA 000000014000eaf0     AccessInfo.obj
 0003:00000b60       ?szAppName@?1???0Jaccesswalker@@QEAA@H@Z@4PADA 000000014000eb60     jaccesswalker.obj
 0003:00000b70       ?szMenuName@?1???0Jaccesswalker@@QEAA@H@Z@4PADA 000000014000eb70     jaccesswalker.obj
 0003:00000c90       logFP                      000000014000ec90     AccessBridgeDebug.obj
 0003:00000ca0       ?retbuf@?1??printError@@9@4PADA 000000014000eca0     AccessBridgeDebug.obj
 0003:00000db0       ?datebuf@?1??getTimeAndDate@@YAPEADXZ@4PADA 000000014000edb0     AccessInfo.obj
 0003:00000e50       GS_ExceptionRecord         000000014000ee50     MSVCRT:gs_report.obj
 0003:00000ef0       GS_ContextRecord           000000014000eef0     MSVCRT:gs_report.obj
 0003:000013d0       ?is_initialized_as_dll@@3_NA 000000014000f3d0     MSVCRT:utility.obj
 0003:000013d1       ?module_local_atexit_table_initialized@@3_NA 000000014000f3d1     MSVCRT:utility.obj
 0003:000013d8       ?module_local_atexit_table@@3U_onexit_table_t@@A 000000014000f3d8     MSVCRT:utility.obj
 0003:000013f0       ?module_local_at_quick_exit_table@@3U_onexit_table_t@@A 000000014000f3f0     MSVCRT:utility.obj
 0005:000001d0       $R000000                   00000001400111d0     jaccesswalker.exe.res
 0005:00000518       $R000348                   0000000140011518     jaccesswalker.exe.res
 0005:000005a8       $R0003D8                   00000001400115a8     jaccesswalker.exe.res
 0005:00000638       $R000468                   0000000140011638     jaccesswalker.exe.res
 0005:000006d8       $R000508                   00000001400116d8     jaccesswalker.exe.res
